:100000000C94FD1F0C94C8200C94C8200C94C8209C
:100010000C94C8200C94C8200C94C8200C94C820C0
:100020000C94C8200C94C8200C94C8200C94C820B0
:100030000C94C8200C946A370C94C8200C94C820E7
:100040000C94C8200C94C8200C94C8200C94C82090
:100050000C94C8200C94C8200C94C8200C94C82080
:100060000C94C8200C94C8200C94C8200C94C82070
:100070000000000000000000000000000000000080
:100080000000000000000000000000000000000070
:100090000000000000000000000000000000000060
:1000A0000000000000000000000000000000000050
:1000B0000000000000000000000000000000000040
:1000C00000000049000000495252000052525C2DCD
:1000D0000000000000000000000000000000000020
:1000E0000040000000494A52004952525B1C5253E2
:1000F0001C25241B2425251B0A0A2D1C12120A0A62
:100100000000000000000000404949494949525B95
:100110005B5B525B1C1C1312241C12090909120997
:100120000909090A0A0A0A0A0A13120A0A12130A10
:100130000000000000009252525252521312130952
:10014000001C0A1212401B65090A0009241B120038
:1001500000251C1C010025241C1C0024252424240B
:100160000000000000005249494000001B135249A2
:100170004900641C1C5B4A481C651C2552491C1C18
:10018000652464491C1C652564491C1C6D2E5C4952
:100190000000000000000000000000490000000016
:1001A000535200000053522500004A5225250000FA
:1001B0005B251300005B53000A1C095B1C657F373D
:1001C0004052522E2E1C525C2E251B1324251C1C23
:1001D00012002525120000121B0000132E37001BF1
:1001E00037372E2E37372E2E2E2E2E2E6E6E6E1C5D
:1001F0001313120009131200001213130012251C0E
:1002000013132E371C131313361C131B1B1B251320
:100210001C1C1B1B1B1C1C1C1C1C1C1C1C1C1C132A
:100220001312121313001313131C000913131C01D0
:100230000037131C13002E2E1C1C001C772E2500CB
:10024000137F251C010A37241C1C0A2E25250900B2
:10025000132E242525252E252525252525252D2E3E
:10026000251B2E2E251C1325251C1C1C1C011C1CAB
:100270001300011C0A000165775C016E7F6E521B42
:1002800025256D1C524925251C1353001C1C1C528E
:100290004A001B135B5B000009525C0000005B5CC2
:1002A000000000001B000000000000000000000033
:1002B000135B7F776E6E136577766E6E1B65777650
:1002C00076761B5BBF76B67609136DBFB7B6001B9B
:1002D000125C76BF0000121B125B00000000090ACE
:1002E0006E6E6E77241C6E6E77251C1C6E776E1CEE
:1002F0001C1C76761C1C2425B765646D6D1B766D01
:100300006D5B09125B5C5B125B641213131B1212B0
:100310001C1C1C1C1C241C1C242525242425251BDA
:1003200000002513000064BF00096EBFBF6D6EBFE3
:100330006D5B12135B12131209000901000000002B
:100340002E1C0900096E010009767F7F12777F7FDE
:100350006412BF775B121B095B121B0900001B09AB
:10036000000000000000000000000000000000008D
:100370007F7F5313130064121B0100001B12000047
:10038000000000000000000000000000000000006D
:10039000000000000000000000000000000000005D
:1003A0000000000000002600000026002F000000D2
:1003B0002F00370000003700FF000000FF00BF00E3
:1003C0000000BF00370000370000002626000000B4
:1003D000000000000000262626262600000000005F
:1003E0002F000000003700000000FF00000000BFE9
:1003F0000000000037000000000026262626260008
:100400000000000000002626262626002F000000FF
:100410000000370000000000FFFFFFFF0000BF00EA
:1004200000000000370000000000262626262600D7
:100430000000000000002626262600002F000000F5
:100440002F00370000003700FFFFFFFF0000BF0054
:100450000000BF00370000003700262626260000D7
:10046000000000000000000026262600002F0000EB
:100470002F00370000003700FF000000FF00BF0022
:100480000000BF00370000370000262626000000CD
:100490000000000000002600000026002F000000E1
:1004A0002F000037003700000000FF00000000BFF1
:1004B00000BF0000370000003700260000002600C3
:1004C000000000000000000000000000000000002C
:1004D000000000000000000000000000000000001C
:1004E0000000009B000000529BA400005B9B6D7706
:1004F00000000000000000000000000000000000FC
:10050000005B000000E4F6FF099BEDF6FFBFA4AD21
:10051000BFBFBFBF767F7FB7B7BF7F766EB7B7BFAE
:1005200000000000000000005BB6F6F6F6FFFFFFDB
:10053000FFBFFFFFFFBFBFAEFFFFFFB7AD65FFFF10
:10054000B7B6AD65FFFFBFB7AE6EFFFFBFB7B7650C
:10055000000000000000F6F6EDEDADA4B66D6D5C98
:10056000526E6565655265765C5C52536E246552C9
:10057000526E25255B52772D2525526E6E2D252531
:10058000000000000000A49B9B4900006564A49B40
:1005900092006D2525649349656E652E9B52242536
:1005A0006D25655225246D2D655225256E2E6452CC
:1005B00000000000000000000000004A00000000F1
:1005C0005B9B0000005B5B2D0000525B2E2E000148
:1005D0005B2D1C01005C5B014A654A5B1C6E7F77EA
:1005E000495B9B77776D5B65776E65656D2D25251E
:1005F0005C522E25130949641C09095C7F7F091C84
:100600007F7F777F777F77777F7F7776777F7F6E44
:10061000656E6EA4B6FF655BA4B7BFFF526DBFBF2A
:10062000BFFF7FBFBFBFBFFFBFBFB7BFFFFF7FB76A
:10063000BFBFFFFF6EB7BFBFFFFF77BFBFBFFFFFEB
:10064000FFFFBFBFB75BFFFFBFBFA464FFFFBFAD2E
:10065000A47FFFFFBFA4BF7FFFBFADBFBFBFFFB67B
:10066000BFBFBF77F7BFBFBF7777FFBFBFBF6452C2
:100670006D7F6E2E2D2D7F766E6E6E2E7777777650
:100680002E1C7F776E251C25776525251C096E6E2F
:100690001C0949255B494A6E7F645377BF775B5CD1
:1006A000256E6E255B4A25651C1B5B002524245B9B
:1006B00053001C1B5B5C00000A5B64000000646468
:1006C000000000005C0000000000000000000000CE
:1006D0005B5C7FBF77765C6D7FB777775C6D7FBF44
:1006E00077775C64BFBFBFBF0A5C6EBFBFBF0065EA
:1006F000646DBFBF00005B6D646D00000000125BA5
:100700007777777F6E6E77777F766D7677BF776D49
:100710006E76BF7F6D6E767FBF7676BFBF76BFBFCA
:10072000BFB664ADADB6B6ADBFFF646DADB6AD647A
:1007300077BFBFBFFFFF77BFBFBFFFFF7FBFBFBF99
:10074000FFF6BFB7ADF6FFFFA4ADFFFFFFFFFFFF52
:10075000FFFFFFFFFFFFFFF6A4005B520000000059
:10076000BFBFAD5B64BFB6ADADBFFFBFFFFFFFFF57
:10077000BF64FFFFBFB6765BFFBFBF5B0000FF5CDF
:100780000000000000000000000000000000000069
:10079000BFBF645C5C006E5C654900006D5B00007F
:1007A0000000000000000000000000000000000049
:1007B0000000000000000000000000000000000039
:1007C0000600040000000100020003000400050010
:1007D00006000700080009000A000B000C000D00CD
:1007E0000E000F0010000000110012001300140092
:1007F000150016000600030000001700180019007D
:100800001A001B001C001D001E001F0020002100FC
:10081000220023002400250026000000000208001A
:10082000085504085A0000F8000990000A1E320515
:100830000000FF0000001C0800000000883B963B01
:10084000743C1A400640993BA83BB73BEE3FC53B82
:10085000D33B00000001000200030004000501007A
:10086000010101020103010401050200020102026B
:10087000020302040205030003010302030303044D
:100880000305040004010402040304040405050034
:10089000050105020503050405050600060106021B
:1008A00006030604060507000701070207030704FD
:1008B00007050800080108020803080408050900E4
:1008C000090109020903090409050A000A010A02CB
:1008D0000A030A040A050B000B010B020B030B04AD
:1008E0000B050C000C010C020C030C040C050D0094
:1008F0000D010D020D030D040D050E000E010E027B
:100900000E030E040E050F000F010F020F030F045C
:100910000F05100010011002100310041005110043
:10092000110111021103110411051200120112022A
:10093000120312041205130013011302130313040C
:1009400013051400140114021403140414051500F3
:1009500015011502150315041505160016011602DA
:1009600016031604160517001701170217031704BC
:1009700017051800180118021803180418051900A3
:10098000190119021903190419051A001A011A028A
:100990001A031A041A051B001B011B021B031B046C
:1009A0001B051C001C011C021C031C041C051D0053
:1009B0001D011D021D031D041D051E001E011E023A
:1009C0001E031E041E051F001F011F021F031F041C
:1009D0001F054F4E4520504C415945520054574F2A
:1009E00020504C4159455253004849474853434FC2
:1009F0005245002D3E000300240137010001130180
:100A00002F0120012CC23B012FF22FC22F322F9237
:100A10002F522F622FA22FE22FD22FB22F720B0351
:100A2000070407050706F809F809F8091E0A0C0A61
:100A3000000AF609F609000A0C0AF609F809F6098F
:100A4000F809F609F8090C0AF609F809F609F8098F
:100A50000E0A120AF809000A0C0A1E0A000AF8090E
:100A6000000A0E0A120A020A120AF809140A080AEF
:100A7000020A020A020A120A0C0AFC091E0AF809F2
:100A8000F609000A1E0A1A0A020A020A120A1E0AB5
:100A9000F8090C0A000AFC090C0A000AFC09000A01
:100AA000FC09140A100A000A0C0A140A100A0C0A9B
:100AB0001E0AF6091E0A0C0A0C0AF609FC09140A99
:100AC000020A020A020A100AF809F6090C0A000AC8
:100AD000F6090E0A0A0A020A080A020A020A160A95
:100AE000020A100AF609F8091A0A100AF8090E0A89
:100AF000020A120AFC090C0A0E0A020A020A080A71
:100B00000A0A0A0A0A0A0A0A0A0A0A0A080A0A0A47
:100B1000020A020A120AF6090C0AF6091E0A0E0A4D
:100B2000120AF609F809000A0C0AF809200A220A32
:100B3000240A0C0AFC090C0A1E0AFC09F6090C0A14
:100B4000FC09FC09FC09FC09FC09FC090C0AF80970
:100B5000F6091E0A0C0A000A0C0AF809F809000A2C
:100B60000C0AF809F6090A0A080A020A120A140A03
:100B7000020A1C0AFC09F809F609F8091E0A0C0AFF
:100B80001E0A000A000A000A000A1E0A0C0AF809D6
:100B9000F6091E0A1A0A020A1C0AF809F8091E0AAE
:100BA0000C0AF609F809000A0C0AFC090E0A1C0ACC
:100BB0001E0A0C0A000AFC09F809140A020A1C0A97
:100BC000F609F809F809F809140A0A0A1C0A140AAD
:100BD000020A020A100AFC090C0A000A000AFC09AF
:100BE0000C0AFC09F609F8091A0A020A020A080A9C
:100BF000020A180A120AFC09140A100AF6090C0A59
:100C0000FC09200A220A240A0C0A1E0A0C0A0C0AF1
:100C1000000A000AF609F8091A0A0A0A0A0A160A54
:100C2000180A0A0A020A000A0C0A1E0AF8090C0A23
:100C3000FC09000A0C0AF6090C0AF8091E0A0C0A3B
:100C40001E0A140A020A020A100AF8090C0A0C0AFF
:100C5000000A000AF609F8090C0AF809F8090C0A52
:100C6000000AF609000A020A1C0AF809F8090C0A27
:100C7000000A1E0A0C0AFC090C0AF609FC091A0AE9
:100C8000020A1C0A1E0A000AFC09000A0C0A0E0AC3
:100C9000020A020A120AFC090C0AF809F8090C0AED
:100CA000F609F809F609000A0C0A000A140A100AE3
:100CB000FC09000A0C0AFC090C0AF609FC090C0ADA
:100CC000FC090C0AF809F809F609000A0C0AF809E7
:100CD000F6091E0A0C0AFC091A0A0A0A0A0A180A64
:100CE000120A000AF809F8090C0A1E0A0C0AF80987
:100CF000F609FC090C0AFC091A0A020A020A1C0A73
:100D0000FC090C0AFC09FC09FC09FC090C0AF8099D
:100D1000F6091E0A0C0A000A0C0A200A220A240AF2
:100D20000C0A000AF6091E0A1A0A020A1C0A000A1C
:100D3000F609F6090C0A000A0C0AF609000A1A0A52
:100D40000A0A180A0A0A020A160A020A180A160ADF
:100D5000020A020A100AF6090C0A1E0A1E0A1E0AD4
:100D60000C0AF809F809FC090C0AF8090C0AFC0934
:100D7000F609F8091A0A020A180A020A020A1C0AE3
:100D8000000A1E0AF809F6090C0A1E0AFC091A0ACA
:100D90000A0A0A0A120AFC091A0A020A020A020AC2
:100DA0001C0AF609000A0A0A100AF6091A0A020AB7
:100DB000160A020A1C0AF609F809FC09F6090C0AC7
:100DC000FC09F809FC09F8091A0A020A020A100AC1
:100DD000F809F8090E0A160A100A000AF809000AAA
:100DE0000C0A000AF809F809000AFC090C0AF809BB
:100DF0000C0A1E0A1A0A020A020A020A020A1C0A3B
:100E0000000AF609F8091E0A0C0AF609FC09F60997
:100E1000000AF6091E0A0C0A1E0AF809000AF80957
:100E20000C0AF809F60902020405070603030F106D
:100E300011121314151617020318191A1B1C1D067C
:100E40000120211E1F222306042425262728292AC3
:100E50002B2C2D2E2F30313232333435363232377F
:100E60003806033032393A323435323B3C3238308E
:100E7000323D3E3234150408070000000000170020
:100E800000000000000000000000000005060D0F3B
:100E9000111312160F1A0D0F110F0E0F190D0F0D42
:100EA0000A03040C0C0C140C0C0C17160B0C0C0D78
:100EB000180C0C0C0C000201090B100010150B1083
:100EC000090A1010090B10090B100018111010114D
:100ED00018101810111810111118111018101810DE
:100EE00010111111111011101118181110101018E3
:100EF00010101811181118111811101111101011CB
:100F000018181811111011101810181110181011AC
:100F100010181811111011111811101011181111A9
:100F200011111011111818111010101011101110AA
:100F3000101110101111101811111011181811188A
:100F40001110111110181811181010111110111181
:100F50001011101810181118181111111818111853
:100F60001110111110181810111111101111101861
:100F70001010111118101810101111111018111152
:100F80001811101111181010181011181011111833
:100F90001011111000000010180000525211100022
:100FA00052525210000052525210005252525218D5
:100FB000005252525211000952525210181111107F
:100FC0001800000010111193930000181052529352
:100FD00000101152525200001052525293001052FF
:100FE000525293001852525293001152525293008F
:100FF00018525252520011525252930010525252F1
:1010000052001152525252001011101018101010AC
:1010100010181010181011111010111800525252FF
:1010200052110009525252100052525252110009EC
:10103000525252100009525252101018101011182A
:101040001010181010111010111110105B525B527B
:1010500009111052095B091811095B5B5211100943
:101060005B095210095B5B5B5B110952095B521013
:10107000105B09525211520952525B095B525B528A
:1010800010525B520910185252095B11105B520941
:101090005B11115B095B5B5B10520952091011096E
:1010A000525B0911185B52095252110910115B1061
:1010B00009525B52095B095252095B5B525B520950
:1010C0005B09525B095B5B5B5B520952095B52092E
:1010D000525B0952525B520952525B095B525B529E
:1010E00009525B52095B095252095B5B525B520920
:1010F0005B09525B095B5B5B5B520952095B5209FE
:1011000052181152525B101110185B095B525B525E
:1011100009525B52095B095252095B5B525B5209EF
:101120005B09525B095B5B5B5B520952095B5209CD
:10113000525B0952525B520952525B0000000000A0
:10114000000000000000000000000000000000009F
:10115000000000000000000000000000000000008F
:10116000000000000000000000000000000000007F
:101170000000000000000000000000000000141447
:1011800014000000141414000000141414000014BF
:1011900014141414000000000000001811101011A5
:1011A0000010181011001011111811001010181053
:1011B0001000101111101100101818110010101843
:1011C000100019101011000819201000100000184C
:1011D00019190010190000201910192019201920C0
:1011E000192020201920181919201820182018104B
:1011F000181919191918101919191819181010187F
:1012000019000010181910192000101019191900D0
:1012100000181819191819001818181018080019AA
:1012200019102018001919102018000008101010AB
:1012300018000810101818180010101810180010B6
:1012400010101911001019181900081010101008AA
:10125000091018101010080818101020181019196B
:101260001810101910191919101920191919101915
:1012700020191919101918181918101918191910F6
:101280001819191018101820181910191919180000
:1012900010191919180010182019202000201918E9
:1012A000181800181819191000181919200800200A
:1012B0001919101000201919192000081010181001
:1012C00010081019181819110819101819080819F8
:1012D0001818190808100811101808081010181903
:1012E00008081010181819080808101919201818DB
:1012F000101919191918101910191818201018197F
:1013000010102011181010111810181011101908B1
:1013100010111111101008180808101819201919A7
:101320000019101819200020101919200020102071
:101330001919001011181118001119182000101097
:1013400008110800191010080800101811101011C9
:101350001810181011181011111811100010181071
:1013600010110011111000000018181100000018D1
:10137000101018110011181118110011111010116E
:101380001818181111101100181018111000101150
:101390001018180000001111180000001118110099
:1013A000111110111100181110101010111011103E
:1013B000001110101111001811111000001811184F
:1013C0001100151110180015151010110015151128
:1013D0001000141515181100141415001818111800
:1013E0001100111110181800001111101116001819
:1013F00010101115160018101015160010181115E0
:1014000015160011111515160010111800131314DC
:1014100015100013131414001213131314000012E8
:1014200012131300120000121300125B12000000CE
:1014300012125B5B5B00125B1200001515151600A3
:101440001815151516001114151515160014151577
:10145000150000141500005B000000AD5BAD005BE3
:10146000AD5BADAD000000AD5BAD000012125B00E6
:101470006D00125B12006D00120000006D00120082
:101480006D6D6D00120000006D00125B12006D00AA
:1014900012125B006D00125B12006D6D005BADAD52
:1014A000006D00AD5BAD006D000000AD006D6D6DB9
:1014B00000AD006D000000AD006D00AD5BAD006DD6
:1014C000005BADAD006D00AD5BAD001011101110F3
:1014D0000011101011110018111110001618111818
:1014E0001100151110180015151010110014151108
:1014F00010001314151811001313141118181118D3
:1015000011001111101818001111111011160018E6
:1015100010101116001018101015160010181115C3
:1015200016001011111515160010111011101110C0
:10153000101110101111101811111011001811189C
:1015400011100011101818001510101111001411AD
:101550001011001314181118001313001818111883
:101560001100001110181816001111101115160095
:101570001010111516001810101515160018111559
:10158000151600111114151516001118001212135A
:101590001410000012131311001200001210001298
:1015A0005B0000110012125B5B1800125B125B18EB
:1015B0000012125B5B1100125B125B151516001115
:1015C0001814155200101100005B00111000ADAD91
:1015D000001818AD5BAD0011185BADAD001811AD72
:1015E0005BAD0011115BADAD0010100012125B007D
:1015F0006D00125B12006D0012125B006D00125B39
:101600001200000012125B125B00125B125B5B00A7
:1016100012125B125B00125B125B5B6D005BADAD87
:10162000006D00AD5BAD006D005BADAD000000ADC9
:101630005BAD005BAD5BADAD00AD5BAD5BAD005BCD
:10164000AD5BADAD00AD5BAD5BAD0018110012122E
:1016500013101800001213111100120000101800CE
:10166000125B0011110012125B181800125B1218A5
:10167000100012125B111800125B121415151600DF
:10168000181314155200111200005B00100000AD79
:10169000AD00185BAD5BAD00185B5BADAD00115BE1
:1016A000AD5BAD00115B5BADAD0010100012125BC5
:1016B0005B1100125B12AD1800ADAD5BAD180012EE
:1016C0005BAD5B11005BADADAD1000AD125BAD115C
:1016D00000ADAD5BAD1800125BAD5BAD5BAD00184E
:1016E000115BADAD000000AD5BADAD5BAD5BAD5B67
:1016F0005BAD5BADADADADADAD5BADAD5BADADAD62
:101700005BADAD5BAD5BAD5B5BAD5B0012125B12C5
:10171000AD00125B12AD5BAD5BADAD5BAD5BAD5BC8
:101720005BAD5BADADADADADAD5BADAD5BADADAD31
:101730005BADAD5BAD5BAD5B5BAD5B5BAD5BADAD69
:1017400000AD5BADADAD00AD5BADAD5BAD5BAD5BBD
:101750005BAD5BADADADADADAD5BADAD5BADADAD01
:101760005BADAD5BAD5BAD5B5BAD5B1011001212B1
:101770005B000000125B5BAD5BADAD5BAD5BAD5B79
:101780005BAD5BADADADADADAD5BADAD5BADADADD1
:101790005BADAD5BAD5BAD5B5BAD5B5BAD5BAD00B6
:1017A00011AD5BADAD0018AD5BADAD00115BAD5BD8
:1017B000AD0011ADADADAD00105BADADAD0011AD87
:1017C0005BADAD00115BAD5BAD001118005BADAD65
:1017D000AD1000AD125BAD1100ADAD5BAD100012F0
:1017E0005BAD5B11005BADADAD1800AD125BAD182C
:1017F00000ADAD5BAD1100125BAD5BADADADADADA0
:10180000AD5BADAD5BADADAD5BADAD5BAD5BAD5BF4
:101810005BAD5BADADADADADAD5BADAD5BADADAD40
:101820000000AD5BAD00000000AD5BADADADADAD9A
:10183000AD5BADAD5BADADAD5BADAD5BAD5BAD5BC4
:101840005BAD5BADADADADADAD5BADAD5BADADAD10
:101850005BADAD5BAD5BAD5B5BAD5BADADADADADA4
:10186000AD5BADAD5BADADAD5BADAD5BAD5BAD5B94
:101870005BAD5BADADADADADAD5BADAD5BADADADE0
:101880005BAD0000AD5BAD00000000ADADADAD00E7
:10189000185BADADAD0011AD5BADAD00105BAD5BE8
:1018A000AD0018ADADADAD00185BADADAD0011AD87
:1018B0005BADAD00115BAD5BAD001010005BADAD7D
:1018C000AD1100AD125BAD1800ADAD5BAD180012EF
:1018D0005BAD5B11005BADADAD1000AD125BAD114A
:1018E00000ADAD5BAD1800125BAD5B00000000AD5C
:1018F000AD00000000ADAD000000005BAD000000D9
:1019000000AD5B00000000ADAD00000000ADADAD6E
:101910005BADAD5BAD5BAD5B5BAD5BADAD000000EA
:10192000005BAD00000000AD5B000000005BAD009F
:10193000000000ADAD000000005BAD00000000AD98
:101940005BADAD5BAD5BAD5B5BAD5BADADADAD0060
:10195000115BADADAD0018AD5BADAD00115BAD5B26
:10196000AD0011ADADADAD00105BADADAD0011ADD5
:101970005BADAD00115BAD5BAD0011ADADADADAD1F
:10198000AD5BADAD000000AD5BAD0000005BAD0038
:101990001B001BADAD001B001BAD001B1B001BADD6
:1019A000001B1B001B5B001B1B001BADADADADADD9
:1019B000AD0000005BADAD000000AD5BAD1B001BDA
:1019C00000AD5B1B001B00ADAD1B001B1B00AD1B66
:1019D000001B1B00AD1B001B1B005BAD00001B00B0
:1019E0001B001B001B001B001B001B001B0000003A
:1019F000000000001B001B001B001B001B001B0045
:101A00001B001B001B001B001B001B1B001B0000FE
:101A1000AD1B001B001B001B001B001B0000000077
:101A20000000001B001B001B001B001B001B001BF9
:101A3000001B001B001B001B001B00001B001B00E9
:101A40001B001B001B001B001B001B001B001B00BE
:101A50001B001B000000000000001B001B001B00FF
:101A60001B001B001B0000000000001B001B001BD4
:101A7000001B001B001B001B001B001B001B001B8E
:101A8000001B000000000000001B001B001B001BCF
:101A9000001B001B000000000000005200000000BE
:101AA000005252030303035B5B05050505ADAD075B
:101AB0000707075B5B050505055B5B05050505522B
:101AC0005203030303520000000000000000050061
:101AD00000000004030400000304230305040405BC
:101AE000040303000323242304030025230300002D
:101AF0000423030500000324260300009DBDBD9DB3
:101B0000000003BDBD03000007BDBD070000AD0020
:101B100000AD002D9D12129D2D2D2D2D2D2D2D2D25
:101B2000002D2D002D2D002D2D002D101110000049
:101B30001011020300001018020303041818020316
:101B4000030411110203030418100203030411110A
:101B500002030304101811181811110000000000EE
:101B60000000000000000000000000000000000075
:101B70000000000000000000000000000000000065
:101B80000000000000000000000000040404040243
:101B9000000F0F0F0F03000F0F0F0F04000F0F0F99
:101BA0000F04000F0F0F0F04000F0F0F0F04000F93
:101BB0000F0F0F030004040404020000050F0F0FB1
:101BC0000F00050F0F0F0F00050F0F0F0F00050F70
:101BD0000F0F0F00050F0F0F0F00050F0F0F0F0056
:101BE000040F0F0F0F00030404040400000002069A
:101BF0000F00000105060F0000020F0F0F00000389
:101C00000F0F0F0000030F0F0F0001030F0F0F0046
:101C100002040F0F0F0004050F0F0F0F0500000047
:101C200000060300000000030100000000020000A5
:101C3000000000020000000000020000000000039D
:101C40000000000000020000000000000000000092
:101C50000000000000000000000000000100000083
:101C60000000030000000000040000000000040069
:101C7000000000040600000000060F01050F0F051C
:101C80000001050F0F050004060F0F0400060F0FDB
:101C90000502000F0F0F0300000F0F060200000FD8
:101CA00006040100000F0501000000030303030206
:101CB000000F0F0F0F03000F0F0F0F04000F0F0F78
:101CC0000F04000F0F0F0F04000F0F0F0F04000F72
:101CD0000F0F0F04000F0F0F0F0400000204040485
:101CE0000400030F0F0F0F00040F0F0F0F00040F5E
:101CF0000F0F0F00040F0F0F0F00040F0F0F0F0037
:101D0000030F0F0F0F0002040404040001060F0666
:101D1000030000040F0F0F0000020F0F0F00000060
:101D20000F0F0F000000020F0F000000000506005B
:101D300000000000020000000000000000000000A1
:101D4000000202010000000F0F030000000F0F034C
:101D50000000000F0F030000000F0F03000000033E
:101D60000302000000000000000000030F0F060146
:101D7000000F0F0F0400000F0F0F0200000F0F0FD6
:101D80000000000F0603000000060401000000022E
:101D9000010000000001000000000000050F0F0519
:101DA0000000050F0F050000050F0F050000050FCF
:101DB0000F050000050F0F050000050F0F050000BF
:101DC000050F0F050000050F0F05000000000000C3
:101DD00000000000000002000000000F0F000000E3
:101DE000030F0F0000000F0F0F0000020F0F0F0076
:101DF00000040F0F0F0001060F0602000000000094
:101E000000000000010202000000030F0F000000AC
:101E1000030F0F000000030F0F000000030F0F005F
:101E200000000203030000000000000100000000A9
:101E3000000200000000000F05010000000F060373
:101E40000000000F0F0F0000000F0F0F0200000F27
:101E50000F0F040000020F0F06010000050F0F0511
:101E60000000050F0F050000050F0F050000050F0E
:101E70000F050000050F0F050000050F0F050000FE
:101E8000050F0F050000030303030000010505050E
:101E90000100050F0F0F0400050F0F0F0F00050FB6
:101EA0000F0F0F00050F0F0F0F00050F0F0F0F0083
:101EB000050F0F0F0F00050F0F0F05010505050199
:101EC00000040F0F0F05000F0F0F0F05000F0F0F6E
:101ED0000F05000F0F0F0F05000F0F0F0F05000F5D
:101EE0000F0F0F0500050F0F0F0500000000000089
:101EF00000030000000002050000000003050000D0
:101F00000000030603000003050F0F0000050F0F7C
:101F10000F0000050F0F0F0303060F0F0F0F0F0F1A
:101F20000F0F0F0F0F0F0F0F0F0F0F0F0F00050FDA
:101F30000F0F0000050F0F0F0000050F0F0F00001F
:101F4000000000000000000000000000050F0F0569
:101F50000000050F0F060200050F0F0F0F00050F01
:101F60000F0F0F00050F0F0F0F00050F0F0F0F00C2
:101F7000030303030300000000000000050F0F052A
:101F80000000050F0F060200050F0F0F0F00050FD1
:101F90000F0F0F00050F0F0F0F00050F0F0F0F0092
:101FA000050F0F060300050F0F05000003030303D1
:101FB0000000050F0F050000050F0F050000050FBD
:101FC0000F050000050F0F050000050F0F050000AD
:101FD000050F0F050000050F0F050000050F0F0589
:101FE0000002060F0F05000F0F0F0F05000F0F0F58
:101FF0000F05000F0F0F0F05000F0F0F0F05000348
:10200000060F0F050000050F0F0500000303030373
:102010000000050F0F050005050F0F05050F0F0F39
:102020000F0F0F0F0F0F0F0F0F05050F0F050500F7
:10203000050F0F050000050F0F0500000000000050
:1020400000000F0F0F0F00000F0F0F0F0000050F04
:102050000F0F0000050F0F0F0000050F0F0F0000FE
:102060000000000000000000000000FF0000000071
:1020700000FF0000000000FF00FFFF0000FF00FF66
:1020800000FF00FF00FF00FF00FF00FF00FF000057
:102090000000000000000000000000000000000040
:1020A0000000000000000000FF00FF000000FF0033
:1020B000FF00FF00FF00FF00FF0000FF0000000026
:1020C00000FF00000000FF00000000000000000012
:1020D00000000000000000FF0000FF00FF00FF0004
:1020E000FF00FF00FF00FF00FFFF000000FF0000F7
:1020F00000000000000000000000000000000000E0
:102100000000000000000000FFFF00000000FF00D2
:102110000000FF00FF000000FF00FF0000000000C3
:1021200000000000000000000000FF0000000000B0
:1021300000000000000000FFFF00FFFF0000FF00A4
:10214000FF000000FF00FF0000FFFF00FF00000095
:10215000FF00000000FFFF00000000000000000082
:1021600000000000000000FFFF0000FF000000FF73
:1021700000FF00FF00FF0000FF00FFFF0000FF0066
:10218000000000000000000000000000000000004F
:1021900000000000000000FF0000FF0000FF00FF43
:1021A00000FF000000FF000000000000FFFF000033
:1021B000000000000000000000000000000000001F
:1021C00000000000000000FF00FF00FFFFFF00FF15
:1021D000000000FF00FF00FF0000FF000000FF0004
:1021E000FF00000000FF00000000000000000000F1
:1021F000000000000000000000FFFF0000FF00FFE3
:102200000000FFFF00FF0000FFFF00FF00000000D4
:10221000000000000000000000000000FF000000BF
:102220000000FF00000000FFFF0000FFFF00FF00B4
:10223000FF000000FF000000FFFFFF00FFFF0000A5
:102240000000000000000000000000000000FF008F
:1022500000000000FF0000000000FF00FF00000081
:10226000FFFF00000000FF00FFFF0000FF00FFFF76
:10227000000000000000000000000000FF00FF0060
:10228000FF000000FF00FF00FF00FF00FF00FF0055
:10229000FF00FF00FF00FF00FF00FF00FF00FF0046
:1022A000000000000000000000000000FF0000002F
:1022B0000000000000000000FF00FFFF0000FF0022
:1022C000FF00FF00FF00FF00FF00FF00FF00FF0016
:1022D00000000000000000000000000000000000FE
:1022E000000000000000000000FFFF000000FF00F1
:1022F000FF000000FF00FF00000000FFFF000000E3
:102300000000FF000000FFFF0000000000000000D0
:1023100000000000000000FF00FF0000FFFF00FFC2
:1023200000FF00FF00FF00FF0000FF000000FF00B3
:10233000FF00000000FF000000000000000000009F
:10234000000000000000000000FF00FF00FF00FF91
:1023500000FF00FF00FF00FF00000000FFFF000083
:10236000000000000000000000000000000000006D
:1023700000000000000000FFFF0000FFFFFF000062
:10238000000000FF000000FF00FF000000FFFF0052
:10239000000000000000000000000000000000003D
:1023A00000000000000000FF0000FF0000FF00FF31
:1023B00000FF000000FF00FF00FF0000FF00000022
:1023C000000000000000000000000000000000000D
:1023D00000000000000000FFFFFFFF0000FF00FF03
:1023E00000FF00FF00FF00FF00FF00FF00FF0000F4
:1023F0000000000000000000000000FF000000FFDF
:1024000000FF0000000000FFFF0000FF00FF00FFD2
:1024100000FF00FF00FF00FF00FFFF0000FF0000C3
:1024200000000000000000000000000000000000AC
:102430000000000000000000FF000000FFFF00FFA0
:1024400000FF00FF000000000000FFFF00FFFF0092
:1024500000000000000000000000000000FF00007D
:10246000000000FF000000FF00FF0000000000FF70
:10247000000000FF00000000000000FF000000005E
:10248000000000000000000000000000000000004C
:10249000000000000000000000000000000000003C
:1024A000000000000000000000000000000000002C
:1024B00000000000000000000000000000FF00001D
:1024C0000000FFFFFF000000FFFFFF00000000FF13
:1024D0000000000000FF00000000000000000000FD
:1024E00000FF000000000000000000FFFF00FFFFF1
:1024F00000FFFF00FFFF00FF0000FF0000000000E2
:1025000000000000000000000000000000000000CB
:1025100000000000000000000000000000000000BB
:102520000000FF00FF0000FFFFFFFFFF0000FF00B3
:10253000FF000000FF00FF0000FFFFFFFFFF0000A3
:10254000FF00FF000000000000000000FF0000008E
:102550000000FFFFFF0000FF000000000000FFFF81
:10256000000000000000FF0000FFFFFF000000006F
:1025700000FF000000000000000000FFFF0000FF5F
:1025800000FFFF0000FF00000000FF00000000FF50
:1025900000000000FF00000000FF0000FFFF00FF40
:1025A0000000FFFF0000000000000000FF0000002E
:1025B00000FF00FF000000FF00FF00000000FF0020
:1025C000000000FF00FF00FF00FF0000FF00000010
:1025D000FFFF00FF0000000000000000FFFF000000
:1025E0000000FFFF00000000FF00000000000000EE
:1025F00000000000000000000000000000000000DB
:1026000000000000000000000000000000FF0000CB
:102610000000FF0000000000FF0000000000FF00BD
:1026200000000000FF0000000000FF0000000000AC
:1026300000FF00000000000000000000FF0000009C
:10264000000000FF0000000000FF0000000000FF8D
:102650000000000000FF0000000000FF000000007C
:10266000FF0000000000000000000000000000006B
:102670000000FF00FF000000FFFFFF0000FFFFFF62
:10268000FFFF0000FFFFFF000000FF00FF00000051
:10269000000000000000000000000000000000003A
:1026A000000000FF0000000000FF000000FFFFFF2F
:1026B000FFFF000000FF0000000000FF000000001E
:1026C000000000000000000000000000000000000A
:1026D00000000000000000000000000000000000FA
:1026E00000000000000000000000FFFF00000000EC
:1026F000FFFF00000000FF000000000000000000DD
:1027000000000000000000000000000000FFFFFFCC
:10271000FFFF0000000000000000000000000000BB
:1027200000000000000000000000000000000000A9
:102730000000000000000000000000000000000099
:1027400000000000000000000000FFFF000000008B
:10275000FFFF00000000000000000000000000007B
:102760000000000000FF00000000FF00000000FF6C
:1027700000000000FF00000000FF0000000000005B
:102780000000000000000000000000002F2F2F00BC
:10279000002F0000002F002F00002F2F002F002FF0
:1027A000002F002F2F00002F002F0000002F00000F
:1027B0002F2F2F000000000000000000002F00005D
:1027C00000002F2F00000000002F00000000002F4D
:1027D00000000000002F00000000002F000000009B
:1027E0002F2F2F0000000000000000002F2F2F00CF
:1027F000002F0000002F00000000002F0000002F1D
:102800002F0000002F000000002F00000000002F0C
:102810002F2F2F2F00000000000000002F2F2F006F
:10282000002F0000002F00000000002F00002F2FBD
:102830002F0000000000002F002F0000002F0000DC
:102840002F2F2F00000000000000000000002F00CC
:102850000000002F2F0000002F002F00002F00008D
:102860002F00002F2F2F2F2F000000002F0000001F
:1028700000002F00000000000000002F2F2F2F2F3E
:10288000002F00000000002F00000000002F2F2F5D
:102890002F0000000000002F002F0000002F00007C
:1028A0002F2F2F000000000000000000002F2F003D
:1028B00000002F000000002F00000000002F2F2F2D
:1028C0002F00002F0000002F002F0000002F00001D
:1028D0002F2F2F00000000000000002F2F2F2F2F80
:1028E00000000000002F000000002F000000002F5B
:1028F000000000002F00000000002F00000000007A
:102900002F00000000000000000000002F2F2F000B
:10291000002F0000002F002F0000002F00002F2F9D
:102920002F00002F0000002F002F0000002F0000BC
:102930002F2F2F0000000000000000002F2F2F007D
:10294000002F0000002F002F0000002F00002F2F6D
:102950002F2F00000000002F000000002F000000BB
:102960002F2F000000000000000000000000000009
:102970000000000000000000FFFF00000000FFFF5B
:1029800000000000000000000000FFFF0000000049
:10299000FFFF000000000000000000000000000039
:1029A0000000000000000000FFFF00000000FFFF2B
:1029B00000000000000000000000FFFF0000000019
:1029C000FFFF00000000FF0000000000000000FF0B
:1029D00000000000FF00000000FF00000000FF00FA
:1029E0000000000000FF000000000000FF000000E9
:1029F000000000FF000000000000000000000000D8
:102A000000000000000000FFFFFFFFFF00000000CB
:102A1000000000000000000000FFFFFFFFFF0000BB
:102A2000000000000000000000000000FF000000A7
:102A3000000000FF000000000000FF000000000098
:102A400000FF00000000FF00000000FF0000000089
:102A5000FF0000000000000000000000FFFFFF007A
:102A600000FF000000FF0000000000FF000000FF6A
:102A7000FF00000000FF0000000000000000000058
:102A800000FF00000000000000000000FFFFFF004A
:102A900000FF000000FF00FF00FFFFFF00FF00FF3E
:102AA00000FF00FF00FFFFFF00FF0000000000002C
:102AB000FFFFFF000000000000000000FFFFFF001C
:102AC00000FF000000FF00FF000000FF00FF00000B
:102AD00000FF00FFFFFFFFFF00FF000000FF00FFFF
:102AE000000000FF00000000000000FFFFFFFF00EB
:102AF00000FF000000FF00FF000000FF00FFFFFFDD
:102B0000FF0000FF000000FF00FF000000FF00FFCB
:102B1000FFFFFF000000000000000000FFFFFF00BB
:102B200000FF000000FF00FF0000000000FF0000A9
:102B3000000000FF0000000000FF000000FF000098
:102B4000FFFFFF0000000000000000FFFFFFFF008C
:102B500000FF000000FF00FF000000FF00FF00007A
:102B600000FF00FF000000FF00FF000000FF00FF6B
:102B7000FFFFFF0000000000000000FFFFFFFFFF5D
:102B800000FF0000000000FF0000000000FFFFFF4A
:102B9000FF0000FF0000000000FF0000000000FF39
:102BA000FFFFFFFF00000000000000FFFFFFFFFF2E
:102BB00000FF0000000000FF0000000000FFFFFF1A
:102BC000FF0000FF0000000000FF0000000000FF09
:102BD000000000000000000000000000FFFFFF00F8
:102BE00000FF000000FF00FF0000000000FF00FFEA
:102BF000FFFF00FF000000FF00FF000000FF0000DB
:102C0000FFFFFFFF00000000000000FF000000FFCA
:102C100000FF000000FF00FF000000FF00FFFFFFBB
:102C2000FFFF00FF000000FF00FF000000FF00FFAB
:102C3000000000FF0000000000000000FFFFFF0098
:102C4000000000FF0000000000FF0000000000FF87
:102C50000000000000FF0000000000FF0000000076
:102C6000FFFFFF000000000000000000000000FF68
:102C70000000000000FF0000000000FF0000000056
:102C800000FF00FF000000FF00FF000000FF000049
:102C9000FFFFFF0000000000000000FF000000FF39
:102CA00000FF0000FF0000FF00FF000000FFFF002A
:102CB000000000FF00FF000000FF0000FF0000FF19
:102CC000000000FF00000000000000FF0000000006
:102CD00000FF0000000000FF0000000000FF0000F7
:102CE000000000FF0000000000FF0000000000FFE7
:102CF000FFFFFFFF00000000000000FF000000FFDA
:102D000000FFFF00FFFF00FF00FF00FF00FF0000CB
:102D100000FF00FF000000FF00FF000000FF00FFB9
:102D2000000000FF00000000000000FF000000FFA6
:102D300000FFFF0000FF00FF00FF00FF00FF00009A
:102D4000FFFF00FF000000FF00FF000000FF00FF8A
:102D5000000000FF0000000000000000FFFFFF0077
:102D600000FF000000FF00FF000000FF00FF000068
:102D700000FF00FF000000FF00FF000000FF000058
:102D8000FFFFFF0000000000000000FFFFFFFF004A
:102D900000FF000000FF00FF000000FF00FFFFFF3A
:102DA000FF0000FF0000000000FF0000000000FF27
:102DB000000000000000000000000000FFFFFF0016
:102DC00000FF000000FF00FF000000FF00FF000008
:102DD00000FF00FF00FF00FF00FF0000FF000000F9
:102DE000FFFF00FF00000000000000FFFFFFFF00EA
:102DF00000FF000000FF00FF000000FF00FFFFFFDA
:102E0000FF0000FF0000FF0000FF000000FF00FFC8
:102E1000000000FF0000000000000000FFFFFF00B6
:102E200000FF000000FF00FF000000000000FFFFA7
:102E3000FF000000000000FF00FF000000FF000096
:102E4000FFFFFF0000000000000000FFFFFFFFFF8A
:102E5000000000FF0000000000FF0000000000FF75
:102E60000000000000FF0000000000FF0000000064
:102E700000FF000000000000000000FF000000FF55
:102E800000FF000000FF00FF000000FF00FF000047
:102E900000FF00FF000000FF00FF000000FF000037
:102EA000FFFFFF0000000000000000FF000000FF27
:102EB00000FF000000FF00FF000000FF00FF000017
:102EC00000FF00FF000000FF0000FF00FF00000007
:102ED00000FF000000000000000000FF000000FFF5
:102EE00000FF000000FF00FF00FF00FF00FF00FFE9
:102EF00000FF00FF00FF00FF00FF00FF00FF0000D9
:102F0000FF00FF0000000000000000FF000000FFC5
:102F100000FF000000FF0000FF00FF00000000FFB6
:102F200000000000FF00FF0000FF000000FF00FFA6
:102F3000000000FF00000000000000FF000000FF94
:102F400000FF000000FF00FF000000FF0000FF0086
:102F5000FF00000000FF0000000000FF0000000074
:102F600000FF000000000000000000FFFFFFFF0066
:102F700000000000FF00000000FF00000000FF0054
:102F8000000000FF0000000000FF0000000000FF44
:102F9000FFFFFF00000000000000000000FFFF0036
:102FA0000000FF0000000000FF00000000FFFF0025
:102FB00000000000FF0000000000FF000000000013
:102FC00000FFFF00000000000000000000FFFF0005
:102FD0000000FF0000FF00FF00FFFF00FFFF00FFF9
:102FE0000000FFFF00FFFF00FF00FF0000FF0000E8
:102FF00000FFFF000000000000000000FFFF0000D5
:1030000000000000FF0000000000FF0000000000C2
:10301000FFFF00000000FF0000000000FF000000B4
:10302000FFFF000000000000000000FEFEFEFEFEAC
:10303000FEFEFEFEFEFEFEFEFEFEFEFEFEFEFEFEB0
:10304000FEFEFEFEFEFEFEFEFEFEFEFEFEFEFEFEA0
:10305000FEFEFEFEFEFEFEFEFEFEFEFEFE0101FE8A
:10306000FEFEFE0101FEFEFE01010101FEFEFE6FFD
:103070006FFEFE03036F6F03030301010303036F7E
:103080006F0103036FFE03016F6F6FFEFE0101FE10
:10309000FEFEFE0101FEFEFE01010101FEFE010138
:1030A0000101FE03036F6F03030303030303036FB5
:1030B000030303036F6F03030303FEFEFE0101FE20
:1030C000FEFEFE0101FEFEFE01010101FEFEFE6F9D
:1030D0006FFEFEFEFE6F6FFEFEFE03030303FE01A6
:1030E00001016F03FE01016F6F03FEFEFE0101FE91
:1030F000FEFEFE0101FEFEFE01010101FEFEFE6F6D
:103100006FFEFEFEFE6F6FFEFEFE03030303FEFE78
:10311000036F010101FE036F6F0101FE030303034F
:10312000FEFEFE9898FEFEFEFE9898FEFEFEFE98BD
:103130009898FEFE98980101FEFE98980101FEFE07
:103140000101FEFEFE010101FEFEFEFE030303037C
:10315000FEFEFE9898FEFEFEFE9898FEFEFEFE988D
:1031600098FEFEFEFE9898FEFEFEFE9898FEFEFE7D
:10317000FE0101FEFEFE010101FEFEFE030303034C
:10318000FEFEFE9898FEFEFEFE9898FEFEFE9898C3
:1031900098FEFEFE01019898FE0101019898FEFE3E
:1031A000FEFE0101FEFEFE010101FEFE030103031E
:1031B000FEFEFE0198FEFEFEFE0198FEFEFEFE985B
:1031C0009898FEFE98980101FEFE98980101FEFE77
:1031D0000101FEFEFE010101FEFEFEFE03010303EE
:1031E000FEFEFE0198FEFEFEFE0198FEFEFEFE982B
:1031F00098FEFEFEFE9898FEFEFEFE9898FEFEFEED
:10320000FE0101FEFEFE010101FEFEFE03010303BD
:10321000FEFEFE0198FEFEFEFE0198FEFEFE989860
:1032200098FEFEFE01019898FE0101019898FEFEAD
:10323000FEFE0101FEFEFE010101FEFE030303038B
:10324000FEFEFE9898FEFEFEFE9898FEFEFE989802
:1032500098FEFEFE01019898FEFE01019898FEFE80
:10326000FEFE0101FEFEFEFE010101FE030303035B
:10327000FEFEFE9898FEFEFEFE9898FEFEFEFE986C
:1032800098FEFEFEFE9898FEFEFEFE9898FEFEFE5C
:10329000FE0101FEFEFEFE010101FEFE030303032B
:1032A000FEFEFE9898FEFEFEFE9898FEFEFEFE983C
:1032B0009898FEFE98980101FEFE9898010101FE83
:1032C0000101FEFEFEFE010101FEFEFE03010303FD
:1032D000FEFEFE0198FEFEFEFE0198FEFEFE9898A0
:1032E00098FEFEFE01019898FEFE01019898FEFEF0
:1032F000FEFE0101FEFEFEFE010101FE03010303CD
:10330000FEFEFE0198FEFEFEFE0198FEFEFEFE9809
:1033100098FEFEFEFE9898FEFEFEFE9898FEFEFECB
:10332000FE0101FEFEFEFE010101FEFE030103039C
:10333000FEFEFE0198FEFEFEFE0198FEFEFEFE98D9
:103340009898FEFE98980101FEFE9898010101FEF2
:103350000101FEFEFEFE010101FEFEFE030303036A
:10336000FEFEFE9898FEFEFEFE9898FEFEFEFE987B
:1033700098FEFEFEFE0198FEFEFEFE0198FEFEFE99
:10338000FEFE01FEFEFEFEFE01FEFEFE0303030343
:10339000FEFEFE9898FEFEFEFE9898FEFEFEFE984B
:1033A00098FEFEFEFE9898FEFEFEFE9898FEFEFE3B
:1033B000FE0101FEFEFEFE0101FEFEFE030303030D
:1033C000FEFEFE9898FEFEFEFE9898FEFEFEFE981B
:1033D00098FEFEFEFE9801FEFEFEFE9801FEFEFE39
:1033E000FE01FEFEFEFEFE01FEFEFEFE03010303E5
:1033F000FEFEFE0198FEFEFEFE0198FEFEFEFE9819
:1034000098FEFEFEFE0198FEFEFEFE0198FEFEFE08
:10341000FEFE01FEFEFEFEFE01FEFEFE03010303B4
:10342000FEFEFE0198FEFEFEFE0198FEFEFEFE98E8
:1034300098FEFEFEFE9898FEFEFEFE9898FEFEFEAA
:10344000FE0101FEFEFEFE0101FEFEFE030103037E
:10345000FEFEFE0198FEFEFEFE0198FEFEFEFE98B8
:1034600098FEFEFEFE9801FEFEFEFE9801FEFEFEA8
:10347000FE01FEFEFEFEFE01FEFEFEFEFE0101FE60
:10348000FEFEFE0101FEFEFE01010101FEFEFE6FD9
:103490006FFEFE80806F6F80808001018080806F72
:1034A0006F0180806FFE80016F6F6FFEFE0101FE75
:1034B000FEFEFE0101FEFEFE01010101FEFE010114
:1034C0000101FE80806F6F80808080808080806FAF
:1034D000808080806F6F80808080FEFEFE0101FE14
:1034E000FEFEFE0101FEFEFE01010101FEFEFE6F79
:1034F0006FFEFEFEFE6F6FFEFEFE80808080FE018E
:1035000001016F80FE01016F6F80FEFEFE0101FE72
:10351000FEFEFE0101FEFEFE01010101FEFEFE6F48
:103520006FFEFEFEFE6F6FFEFEFE80808080FEFE60
:10353000806F010101FE806F6F0101FE808080803D
:10354000FEFEFE5B5BFEFEFEFE5B5BFEFEFEFE5BCA
:103550005B5BFEFE5B5B0101FEFE5B5B0101FEFE51
:103560000101FEFEFE010101FEFEFEFE8080808064
:10357000FEFEFE5B5BFEFEFEFE5B5BFEFEFEFE5B9A
:103580005BFEFEFEFE5B5BFEFEFEFE5B5BFEFEFE8A
:10359000FE0101FEFEFE010101FEFEFE8080808034
:1035A000FEFEFE5B5BFEFEFEFE5B5BFEFEFE5B5B0D
:1035B0005BFEFEFE01015B5BFE0101015B5BFEFE4B
:1035C000FEFE0101FEFEFE010101FEFE8001808083
:1035D000FEFEFE015BFEFEFEFE015BFEFEFEFE5BEE
:1035E0005B5BFEFE5B5B0101FEFE5B5B0101FEFEC1
:1035F0000101FEFEFE010101FEFEFEFE8001808053
:10360000FEFEFE015BFEFEFEFE015BFEFEFEFE5BBD
:103610005BFEFEFEFE5B5BFEFEFEFE5B5BFEFEFEF9
:10362000FE0101FEFEFE010101FEFEFE8001808022
:10363000FEFEFE015BFEFEFEFE015BFEFEFE5B5B30
:103640005BFEFEFE01015B5BFE0101015B5BFEFEBA
:10365000FEFE0101FEFEFE010101FEFE8080808073
:10366000FEFEFE5B5BFEFEFEFE5B5BFEFEFE5B5B4C
:103670005BFEFEFE01015B5BFEFE01015B5BFEFE8D
:10368000FEFE0101FEFEFEFE010101FE8080808043
:10369000FEFEFE5B5BFEFEFEFE5B5BFEFEFEFE5B79
:1036A0005BFEFEFEFE5B5BFEFEFEFE5B5BFEFEFE69
:1036B000FE0101FEFEFEFE010101FEFE8080808013
:1036C000FEFEFE5B5BFEFEFEFE5B5BFEFEFEFE5B49
:1036D0005B5BFEFE5B5B0101FEFE5B5B010101FECD
:1036E0000101FEFEFEFE010101FEFEFE8001808062
:1036F000FEFEFE015BFEFEFEFE015BFEFEFE5B5B70
:103700005BFEFEFE01015B5BFEFE01015B5BFEFEFC
:10371000FEFE0101FEFEFEFE010101FE8001808031
:10372000FEFEFE015BFEFEFEFE015BFEFEFEFE5B9C
:103730005BFEFEFEFE5B5BFEFEFEFE5B5BFEFEFED8
:10374000FE0101FEFEFEFE010101FEFE8001808001
:10375000FEFEFE015BFEFEFEFE015BFEFEFEFE5B6C
:103760005B5BFEFE5B5B0101FEFE5B5B010101FE3C
:103770000101FEFEFEFE010101FEFEFE8080808052
:10378000FEFEFE5B5BFEFEFEFE5B5BFEFEFEFE5B88
:103790005BFEFEFEFE015BFEFEFEFE015BFEFEFE2C
:1037A000FEFE01FEFEFEFEFE01FEFEFE808080802B
:1037B000FEFEFE5B5BFEFEFEFE5B5BFEFEFEFE5B58
:1037C0005BFEFEFEFE5B5BFEFEFEFE5B5BFEFEFE48
:1037D000FE0101FEFEFEFE0101FEFEFE80808080F5
:1037E000FEFEFE5B5BFEFEFEFE5B5BFEFEFEFE5B28
:1037F0005BFEFEFEFE5B01FEFEFEFE5B01FEFEFECC
:10380000FE01FEFEFEFEFE01FEFEFEFE8001808049
:10381000FEFEFE015BFEFEFEFE015BFEFEFEFE5BAB
:103820005BFEFEFEFE015BFEFEFEFE015BFEFEFE9B
:10383000FEFE01FEFEFEFEFE01FEFEFE8001808019
:10384000FEFEFE015BFEFEFEFE015BFEFEFEFE5B7B
:103850005BFEFEFEFE5B5BFEFEFEFE5B5BFEFEFEB7
:10386000FE0101FEFEFEFE0101FEFEFE80018080E3
:10387000FEFEFE015BFEFEFEFE015BFEFEFEFE5B4B
:103880005BFEFEFEFE5B01FEFEFEFE5B01FEFEFE3B
:10389000FE01FEFEFEFEFE01FEFEFEFEADBDBDAD66
:1038A000FEFEADBDBDADFE2DBDBDBDBD2D2DADBD65
:1038B000BDAD2D2D2D2D2D2D2D2D2D2D2D2D2DFE57
:1038C000FE2D2DFEFEFEFE2D2DFEFEFE9DBDBD9DA0
:1038D000FEFE03BDBD03FEFE07BDBD07FEFEAD003F
:1038E00000ADFE2D9D12129D2D2D2D2D2D2D2D2D3A
:1038F000FE2D2DFE2D2DFE2D2DFE2DFEFEADBDAD82
:10390000FEFEFE07BDBDFEFEFE03BDBDFEFEFEBD0E
:10391000BDADFEFEFE00BDFEFE2D2D2D2DFEFE2DAD
:103920002D2D2DFEFEFEFE2D2DFEFEFEADBDADFEAF
:10393000FEFEBDBD07FEFEFEBDBD03FEFEFEADBD2F
:10394000BDFEFEFEFEBD00FEFEFEFE2D2D2D2DFE5B
:10395000FE2D2D2D2DFEFE2D2DFEFEFEFE2D59FEE3
:10396000FEFEFE2D59FEFEFEFE5959FEFEFEFE59DC
:103970005959FEFE59595959FEFE59590101FEFE89
:1039800001010101FE010101FEFEFEFEFE2D59FEB8
:10399000FEFEFE2D59FEFEFEFE5959FEFEFEFE59AC
:1039A00059FEFEFEFE5959FEFEFEFE5959FEFEFE70
:1039B000FE0101FEFEFE010101FEFEFEFE2D59FE8E
:1039C000FEFEFE2D59FEFEFEFE5959FEFEFE595921
:1039D00059FEFEFE59595959FEFE01015959FE0181
:1039E00001010101FEFEFE010101FEFEFE592DFE58
:1039F000FEFEFE592DFEFEFEFE5959FEFEFE5959F1
:103A000059FEFEFE59595959FEFE01015959FEFE53
:103A100001010101FEFEFEFE010101FEFE592DFE27
:103A2000FEFEFE592DFEFEFEFE5959FEFEFEFE591B
:103A300059FEFEFEFE5959FEFEFEFE5959FEFEFEDF
:103A4000FE0101FEFEFEFE010101FEFEFE592DFEFD
:103A5000FEFEFE592DFEFEFEFE5959FEFEFEFE59EB
:103A60005959FEFE59595959FEFE59590101FEFE98
:103A70000101010101FE010101FEFEFEFE5959FE98
:103A8000FEFEFE5959FEFEFEFE5959FEFEFEFE598F
:103A900059FEFEFEFE0159FEFEFEFE0159FEFEFE2F
:103AA000FEFE01FEFEFEFEFE01FEFEFEFE5959FE7A
:103AB000FEFEFE5959FEFEFEFE5959FEFEFEFE595F
:103AC00059FEFEFEFE5959FEFEFEFE5959FEFEFE4F
:103AD000FE0101FEFEFEFE0101FEFEFEFE5959FE44
:103AE000FEFEFE5959FEFEFEFE5959FEFEFEFE592F
:103AF00059FEFEFEFE5901FEFEFEFE5901FEFEFECF
:103B0000FE01FEFEFEFEFE01FEFEFE04FEFEFEFEC9
:103B1000FEFEFE04FE04FEFEFEFEFEFEFE0503FEAD
:103B20000303FE0304FE04050504FE03FE05FEFE7A
:103B300003FE03030503FE0303FE0304FEFE05FE6E
:103B400005FE0504FE040405FEFEFEFE050503FE5B
:103B50000303FE0304FE04050504FE03FE05FEFE4A
:103B600003FE03030503050303FE03FEFEFEFEFE44
:103B7000FEFE05FEFEFEFE04FEFEFEFE05FEFEFE51
:103B8000FEFEFE03FEFEFE04FEFEFEFEFEFEFEFE4A
:103B900003FE03FE0503FEFEFEFEFEFEFEFE04FE29
:103BA00005FEFE03FE04FEFE04FE03FEFEFEFEFE18
:103BB00004FEFE04FE03FEFE04FEFE03FEFEFEFE09
:103BC00005FEFEFEFEFEFEFEFEFE050503FE04FEF5
:103BD00005FE0503FE05FE0504FE03FE05FEFEFED2
:103BE00004050504FE03FE050405FE03FE05FEFEB6
:103BF000050505FE0505FEFEFE050505FEFE04FEA7
:103C000004FE04FEFE05FE05FEFEFEFE05FEFEFEB3
:103C100004FEFE04FEFEFEFE0405FEFEFE05FEFEA4
:103C200005FEFEFE0505FEFEFE05FEFEFEFEFEFE98
:103C3000FEFEFEFEFEFEFEFEFE01FEFEFEFEFEFEA1
:103C4000FE01FEFE01FE01FEFEFEFEFEFEFE01FE88
:103C500001FEFEFEFEFEFEFE01FEFEFEFEFEFEFE7E
:103C600003FE03FEFE13FE02FE0702FE04FE23FE19
:103C70002306FEFE05FE05FE23FEFE24FEFE06FED6
:103C800006FEFE03FE03FE0405FEFEFE030401FE27
:103C900003FEFE022423FEFE23FE0304FE04240290
:103CA000040123FE03050305240223030103FEFE92
:103CB000052D02FEFEFEFE2D2DFEFEFE030105FE7D
:103CC000040403230323FEFE07FE0207FEFE230176
:103CD000230223052404FE04FE2301052D0304030F
:103CE000FE2D2DFEFEFE012D2DFE0200020600001F
:103CF000FB00FF00FF0002090000F10400F900FFD3
:103D00000001010007900000E208050000FF00022A
:103D1000080107C80106000100E700FF00010000DC
:103D200007A00000EC0100FE00010100FF000201FD
:103D30000107C80106000100EC00FF0002040000BA
:103D4000F10400F900FF0002010000F100FF000093
:103D5000ED00010602010100FF0000EC000102017C
:103D600007000207FF00010300FF000208000764CC
:103D70000100140500F700FF0002090000F100FF38
:103D80000002020106000100E000FF00020101063E
:103D9000000100E000FF0002080106000100E00051
:103DA000FF0002050106000100E000FF000209011A
:103DB00006000100E000FF0007FF0001090600F116
:103DC0000A07FF0000ED0001060201010707F000ED
:103DD00000ED00010602010100FF0007FF000109DC
:103DE0000000F60207FF0000F100010602010100D9
:103DF000FF0007000402040007FF000990000A28E2
:103E00000000FB01083703030A03040503030A0348
:103E1000040503030A03040503030A03050000FF66
:103E20000007000402040007FF000990000A2800B0
:103E300000FB01084B04030A04040504030A0404FC
:103E40000A04030504040A04030504050000FF0036
:103E500007000402040007FF000990000A28000080
:103E6000FB01085A030305030405030305030405C6
:103E70000303050304050303050304050303050603
:103E8000050000FF0002010007FF0000FB00083CE6
:103E90000104010104010104010104010104010103
:103EA00004010104010104010104010104010305ED
:103EB0000000FF0002010007FF0000FD00083C05B4
:103EC00004050504050504050A050000FF0007991F
:103ED0000001091000F400FF000000EB3C000000AE
:103EE00000000000F33C00000000000000F53C0072
:103EF000000000010000003D000000000000000E76
:103F00003D000000000100001C3D0000000000001A
:103F1000002D3D000000000000003B3D00000000BF
:103F2000000000463D000000000100004E3D000082
:103F30000000010000593D000000000000006A3D43
:103F400000000000000000783D00000000000000BC
:103F5000803D000000000000008B3D0000000000DC
:103F60000000963D00000000000000A13D000000A0
:103F700000000000AC3D00000000010000B73D0063
:103F8000000000010000DA3D00000000000000F128
:103F90003D00000000000000203E00000000000086
:103FA000004F3E00000000000000843E00000000C2
:103FB000000000B33E00000000010000CD3E000004
:103FC000000050415553454400444F55424C452153
:103FD000004D554C54492100494E53414E45210056
:103FE00047414D45204F5645520052455452593F86
:103FF000004D454E553F003E000011241FBECFEF3F
:10400000D0E1DEBFCDBF14BE88E10FB6F894809337
:104010006000109260000FBE11E0A0E0B1E0E4EBA0
:10402000F8EC02C005900D92AC3AB107D9F71DE04B
:10403000A0ECB1E001C01D92AD36B107E1F7F894F4
:10404000E1ECFAE080E090E020E802C021930196E4
:1040500032E08C309307D4F381EC9AE09093CE0C4D
:104060008093CD0C1092CF0CE2EDFCE080E090E06C
:1040700003C0108201963A9684309105D4F381E012
:104080008093F20C8093F30C8093F10C10928100DA
:1040900015BCE0E0F1E080E090E02EEF02C021935B
:1040A000019680399105DCF39093FC0C8093FB0C16
:1040B00080E00E946838E0E6F6E080E090E050EDB5
:1040C00020EC31E041E00EC010821182009719F41B
:1040D0005093620601C01282348323831782408783
:1040E00001963F96823091057CF39093FC0C80936F
:1040F000FB0C91E09093960A8FEF87B984B980E822
:104100008AB98CE081B98BEF82B91092970A86E068
:104110008093980A109285001092840083E0809327
:1041200089008DE88093880089E08093810082E097
:1041300080936F0082E484BD17BC95BD83E88093B3
:10414000B0001092B3009093B10081E185B9109254
:10415000A80A10929B0A10929C0A1092A30A10922D
:10416000A20A1092A70A1092A60A1092FD0C0E94B1
:10417000613A80E00E94423980FF03C084E00E94DF
:104180003F3978940E94423B0E94B4510C94586489
:104190000C940000A937B337C1371537EBEDC8953C
:1041A0000000EA95E1F700C000C04091650650911B
:1041B00066064ABD5BBDC0916B06D0916C0640900F
:1041C0006D0650906E0690906706F0906206E09043
:1041D0006A0670916106672F6770882400EDA02E33
:1041E000A1E8B6E075D00027E101D30108B9F1E0FC
:1041F000E091910A119311931193119311931193DB
:10420000E091920A119311931193119311931193C9
:10421000E091930A119311931193119311931193B8
:10422000E091940A119311931193119311931193A7
:10423000E091950A11931193119311931193119396
:1042400063957395FA94A9F483940FE0809EF0012E
:10425000E05AF94F058016800ABC1BBCC385D48583
:10426000458456849780F280E2847181672F67705D
:1042700008C00000000000000000000009E00A95EE
:10428000F1F7791509F4E20109F4772709F46627B3
:10429000AA9441F0683019F000C000C0A3CF66278F
:1042A000A096A0CFC895C8950E949A374091980AC9
:1042B000405D4093980A11E000919A0A012700930B
:1042C0009A0AE1E0E093990AE2E0E093360008956B
:1042D0002898E091CD0CF091CE0C01912CE0ED3CB2
:1042E000F20721EC3AE00093B30008F0F901E09303
:1042F000CD0CF093CE0C1E01C0907F06D0908006AE
:1043000080E323E036E0D1E040E056E098E00D9114
:10431000099F112D0F71FA01029FE00DF11D02811D
:10432000C081F601089FE00DF11D139FE00DF11D06
:10433000C093910A059009920590099205900992FF
:104340000590099205900992059009920D91099F97
:10435000112D0F71FA01029FE00DF11D0281C08144
:10436000F601089FE00DF11D139FE00DF11DC093B4
:10437000920A05900992059009920590099205907C
:1043800009920D91289A0590099205900992099F2A
:10439000112D0F71FA01029FE00DF11D0281C08104
:1043A000F601089FE00DF11D139FE00DF11DC09374
:1043B000930A05900992059009920590099205903B
:1043C000099205900992059009920D91099F112D6E
:1043D0000F71FA01029FE00DF11D0281C081F6010B
:1043E000089FE00DF11D139FE00DF11DC093940A8D
:1043F00005900992059009920590099205900992FD
:1044000005900992059009920D91099F112D0F7148
:10441000FA01029FE00DF11D0281C081F601089FA3
:10442000E00DF11D139FE00DF11DC093950A05905D
:1044300009920590099205900992059009920590BC
:10444000099205900992E1013D01DE011EEF4AB596
:104450005BB5639FC0013A2F307ECE2DCC0FDD2798
:10446000C057DE4FE991F881C6E0D1E0CC9020E35F
:10447000C29EA395AF71A32B040E151E080E191E24
:104480000994F001C895C895C895C8950591D9902B
:10449000D1120D2D08B9CC900591D990D1120D2DC6
:1044A00008B9C29E0591D990D1120D2D08B9040EFC
:1044B000151E0591D990D1120D2D08B9080E191E9F
:1044C0000591D990D1120D2D08B9A395AF71059121
:1044D000D990D1120D2D08B9A32BF0010591D990D7
:1044E000D1120D2D08B9CC900591D990D1120D2D76
:1044F00008B9C29E0591D990D1120D2D08B9040EAC
:10450000151E0591D990D1120D2D08B9080E191E4E
:104510000591D990D1120D2D08B9A395AF710591D0
:10452000D990D1120D2D08B9A32BF0010591D99086
:10453000D1120D2D08B9CC900591D990D1120D2D25
:1045400008B9C29E0591D990D1120D2D08B9040E5B
:10455000151E0591D990D1120D2D08B9080E191EFE
:104560000591D990D1120D2D08B9A395AF71059180
:10457000D990D1120D2D08B9A32BF0010591D99036
:10458000D1120D2D08B9CC900591D990D1120D2DD5
:1045900008B9C29E0591D990D1120D2D08B9040E0B
:1045A000151E0591D990D1120D2D08B9080E191EAE
:1045B0000591D990D1120D2D08B9A395AF71059130
:1045C000D990D1120D2D08B9A32BF0010591D990E6
:1045D000D1120D2D08B9CC900591D990D1120D2D85
:1045E00008B9C29E0591D990D1120D2D08B9040EBB
:1045F000151E0591D990D1120D2D08B9080E191E5E
:104600000591D990D1120D2D08B9A395AF710591DF
:10461000D990D1120D2D08B9A32BF0010591D99095
:10462000D1120D2D08B9CC900591D990D1120D2D34
:1046300008B9C29E0591D990D1120D2D08B9040E6A
:10464000151E0591D990D1120D2D08B9080E191E0D
:104650000591D990D1120D2D08B9A395AF7105918F
:10466000D990D1120D2D08B9A32BF0010591D99045
:10467000D1120D2D08B9CC900591D990D1120D2DE4
:1046800008B9C29E0591D990D1120D2D08B9040E1A
:10469000151E0591D990D1120D2D08B9080E191EBD
:1046A0000591D990D1120D2D08B9A395AF7105913F
:1046B000D990D1120D2D08B9A32BF0010591D990F5
:1046C000D1120D2D08B9CC900591D990D1120D2D94
:1046D00008B9C29E0591D990D1120D2D08B9040ECA
:1046E000151E0591D990D1120D2D08B9080E191E6D
:1046F0000591D990D1120D2D08B9A395AF710591EF
:10470000D990D1120D2D08B9A32BF0010591D990A4
:10471000D1120D2D08B9CC900591D990D1120D2D43
:1047200008B9C29E0591D990D1120D2D08B9040E79
:10473000151E0591D990D1120D2D08B9080E191E1C
:104740000591D990D1120D2D08B9A395AF7105919E
:10475000D990D1120D2D08B9A32BF0010591D99054
:10476000D1120D2D08B9CC900591D990D1120D2DF3
:1047700008B9C29E0591D990D1120D2D08B9040E29
:10478000151E0591D990D1120D2D08B9080E191ECC
:104790000591D990D1120D2D08B9A395AF7105914E
:1047A000D990D1120D2D08B9A32BF0010591D99004
:1047B000D1120D2D08B9CC900591D990D1120D2DA3
:1047C00008B9C29E0591D990D1120D2D08B9040ED9
:1047D000151E0591D990D1120D2D08B9080E191E7C
:1047E0000591D990D1120D2D08B9A395AF710591FE
:1047F000D990D1120D2D08B9A32BF0010591D990B4
:10480000D1120D2D08B9CC900591D990D1120D2D52
:1048100008B9C29E0591D990D1120D2D08B9040E88
:10482000151E0591D990D1120D2D08B9080E191E2B
:104830000591D990D1120D2D08B9A395AF710591AD
:10484000D990D1120D2D08B9A32BF0010591D99063
:10485000D1120D2D08B9CC900591D990D1120D2D02
:1048600008B9C29E0591D990D1120D2D08B9040E38
:10487000151E0591D990D1120D2D08B9080E191EDB
:104880000591D990D1120D2D08B9A395AF7105915D
:10489000D990D1120D2D08B9A32BF0010591D99013
:1048A000D1120D2D08B9CC900591D990D1120D2DB2
:1048B00008B9C29E0591D990D1120D2D08B9040EE8
:1048C000151E0591D990D1120D2D08B9080E191E8B
:1048D0000591D990D1120D2D08B9A395AF7105910D
:1048E000D990D1120D2D08B9A32BF0010591D990C3
:1048F000D1120D2D08B9CC900591D990D1120D2D62
:1049000008B9C29E0591D990D1120D2D08B9040E97
:10491000151E0591D990D1120D2D08B9080E191E3A
:104920000591D990D1120D2D08B9A395AF710591BC
:10493000D990D1120D2D08B9A32BF0010591D99072
:10494000D1120D2D08B9CC900591D990D1120D2D11
:1049500008B9C29E0591D990D1120D2D08B9040E47
:10496000151E0591D990D1120D2D08B9080E191EEA
:104970000591D990D1120D2D08B9A395AF7105916C
:10498000D990D1120D2D08B9A32BF0010591D99022
:10499000D1120D2D08B9CC900591D990D1120D2DC1
:1049A00008B9C29E0591D990D1120D2D08B9040EF7
:1049B000151E0591D990D1120D2D08B9080E191E9A
:1049C0000591D990D1120D2D08B9A395AF7105911C
:1049D000D990D1120D2D08B9A32BF0010591D990D2
:1049E000D1120D2D08B9CC900591D990D1120D2D71
:1049F00008B9C29E0591D990D1120D2D08B9040EA7
:104A0000151E0591D990D1120D2D08B9080E191E49
:104A10000591D990D1120D2D08B9A395AF710591CB
:104A2000D990D1120D2D08B9A32BF0010591D99081
:104A3000D1120D2D08B9CC900591D990D1120D2D20
:104A400008B9C29E0591D990D1120D2D08B9040E56
:104A5000151E0591D990D1120D2D08B9080E191EF9
:104A60000591D990D1120D2D08B9A395AF7105917B
:104A7000D990D1120D2D08B9A32BF0010591D99031
:104A8000D1120D2D08B9CC900591D990D1120D2DD0
:104A900008B9C29E0591D990D1120D2D08B9040E06
:104AA000151E0591D990D1120D2D08B9080E191EA9
:104AB0000591D990D1120D2D08B9A395AF7105912B
:104AC000D990D1120D2D08B9A32BF0010591D990E1
:104AD000D1120D2D08B9CC900591D990D1120D2D80
:104AE00008B9C29E0591D990D1120D2D08B9040EB6
:104AF000151E0591D990D1120D2D08B9080E191E59
:104B00000591D990D1120D2D08B9A395AF710591DA
:104B1000D990D1120D2D08B9A32BF0010591D99090
:104B2000D1120D2D08B9CC900591D990D1120D2D2F
:104B300008B9C29E0591D990D1120D2D08B9040E65
:104B4000151E0591D990D1120D2D08B9080E191E08
:104B50000591D990D1120D2D08B9A395AF7105918A
:104B6000D990D1120D2D08B9A32BF0010895F001B1
:104B70003196CC9000C000C000C000C00591D99013
:104B8000D1120D2D08B9C29E0591D990D1120D2DCB
:104B900008B9040E151E0591D990D1120D2D08B932
:104BA000080E191E0591D990D1120D2D08B9A395A3
:104BB000AF710591D990D1120D2D08B9A32BF00139
:104BC0000591D990D1120D2D08B9CC900591D990AD
:104BD000D1120D2D08B9C29E0591D990D1120D2D7B
:104BE00008B9040E151E0591D990D1120D2D08B9E2
:104BF000080E191E0591D990D1120D2D08B9A39553
:104C0000AF710591D990D1120D2D08B9A32BF001E8
:104C10000591D990D1120D2D08B9CC900591D9905C
:104C2000D1120D2D08B9C29E0591D990D1120D2D2A
:104C300008B9040E151E0591D990D1120D2D08B991
:104C4000080E191E0591D990D1120D2D08B9A39502
:104C5000AF710591D990D1120D2D08B9A32BF00198
:104C60000591D990D1120D2D08B9CC900591D9900C
:104C7000D1120D2D08B9C29E0591D990D1120D2DDA
:104C800008B9040E151E0591D990D1120D2D08B941
:104C9000080E191E0591D990D1120D2D08B9A395B2
:104CA000AF710591D990D1120D2D08B9A32BF00148
:104CB0000591D990D1120D2D08B9CC900591D990BC
:104CC000D1120D2D08B9C29E0591D990D1120D2D8A
:104CD00008B9040E151E0591D990D1120D2D08B9F1
:104CE000080E191E0591D990D1120D2D08B9A39562
:104CF000AF710591D990D1120D2D08B9A32BF001F8
:104D00000591D990D1120D2D08B9CC900591D9906B
:104D1000D1120D2D08B9C29E0591D990D1120D2D39
:104D200008B9040E151E0591D990D1120D2D08B9A0
:104D3000080E191E0591D990D1120D2D08B9A39511
:104D4000AF710591D990D1120D2D08B9A32BF001A7
:104D50000591D990D1120D2D08B9CC900591D9901B
:104D6000D1120D2D08B9C29E0591D990D1120D2DE9
:104D700008B9040E151E0591D990D1120D2D08B950
:104D8000080E191E0591D990D1120D2D08B9A395C1
:104D9000AF710591D990D1120D2D08B9A32BF00157
:104DA0000591D990D1120D2D08B9CC900591D990CB
:104DB000D1120D2D08B9C29E0591D990D1120D2D99
:104DC00008B9040E151E0591D990D1120D2D08B900
:104DD000080E191E0591D990D1120D2D08B9A39571
:104DE000AF710591D990D1120D2D08B9A32BF00107
:104DF0000591D990D1120D2D08B9CC900591D9907B
:104E0000D1120D2D08B9C29E0591D990D1120D2D48
:104E100008B9040E151E0591D990D1120D2D08B9AF
:104E2000080E191E0591D990D1120D2D08B9A39520
:104E3000AF710591D990D1120D2D08B9A32BF001B6
:104E40000591D990D1120D2D08B9CC900591D9902A
:104E5000D1120D2D08B9C29E0591D990D1120D2DF8
:104E600008B9040E151E0591D990D1120D2D08B95F
:104E7000080E191E0591D990D1120D2D08B9A395D0
:104E8000AF710591D990D1120D2D08B9A32BF00166
:104E90000591D990D1120D2D08B9CC900591D990DA
:104EA000D1120D2D08B9C29E0591D990D1120D2DA8
:104EB00008B9040E151E0591D990D1120D2D08B90F
:104EC000080E191E0591D990D1120D2D08B9A39580
:104ED000AF710591D990D1120D2D08B9A32BF00116
:104EE0000591D990D1120D2D08B9CC900591D9908A
:104EF000D1120D2D08B9C29E0591D990D1120D2D58
:104F000008B9040E151E0591D990D1120D2D08B9BE
:104F1000080E191E0591D990D1120D2D08B9A3952F
:104F2000AF710591D990D1120D2D08B9A32BF001C5
:104F30000591D990D1120D2D08B9CC900591D99039
:104F4000D1120D2D08B9C29E0591D990D1120D2D07
:104F500008B9040E151E0591D990D1120D2D08B96E
:104F6000080E191E0591D990D1120D2D08B9A395DF
:104F7000AF710591D990D1120D2D08B9A32BF00175
:104F80000591D990D1120D2D08B9CC900591D990E9
:104F9000D1120D2D08B9C29E0591D990D1120D2DB7
:104FA00008B9040E151E0591D990D1120D2D08B91E
:104FB000080E191E0591D990D1120D2D08B9A3958F
:104FC000AF710591D990D1120D2D08B9A32BF00125
:104FD0000591D990D1120D2D08B9CC900591D99099
:104FE000D1120D2D08B9C29E0591D990D1120D2D67
:104FF00008B9040E151E0591D990D1120D2D08B9CE
:10500000080E191E0591D990D1120D2D08B9A3953E
:10501000AF710591D990D1120D2D08B9A32BF001D4
:105020000591D990D1120D2D08B9CC900591D99048
:10503000D1120D2D08B9C29E0591D990D1120D2D16
:1050400008B9040E151E0591D990D1120D2D08B97D
:10505000080E191E0591D990D1120D2D08B9A395EE
:10506000AF710591D990D1120D2D08B9A32BF00184
:105070000591D990D1120D2D08B9CC900591D990F8
:10508000D1120D2D08B9C29E0591D990D1120D2DC6
:1050900008B9040E151E0591D990D1120D2D08B92D
:1050A000080E191E0591D990D1120D2D08B9A3959E
:1050B000AF710591D990D1120D2D08B9A32BF00134
:1050C0000591D990D1120D2D08B9CC900591D990A8
:1050D000D1120D2D08B9C29E0591D990D1120D2D76
:1050E00008B9040E151E0591D990D1120D2D08B9DD
:1050F000080E191E0591D990D1120D2D08B9A3954E
:10510000AF710591D990D1120D2D08B9A32BF001E3
:105110000591D990D1120D2D08B9CC900591D99057
:10512000D1120D2D08B9C29E0591D990D1120D2D25
:1051300008B9040E151E0591D990D1120D2D08B98C
:10514000080E191E0591D990D1120D2D08B9A395FD
:10515000AF710591D990D1120D2D08B9A32BF00193
:105160000591D990D1120D2D08B9CC900591D99007
:10517000D1120D2D08B9C29E0591D990D1120D2DD5
:1051800008B9040E151E0591D990D1120D2D08B93C
:10519000080E191E0591D990D1120D2D08B9A395AD
:1051A000AF710591D990D1120D2D08B9A32BF00143
:1051B0000591D990D1120D2D08B9CC900591D990B7
:1051C000D1120D2D08B9C29E0591D990D1120D2D85
:1051D00008B9040E151E0591D990D1120D2D08B9EC
:1051E000080E191E0591D990D1120D2D08B9A3955D
:1051F000AF710591D990D1120D2D08B9A32BF001F3
:105200000591D990D1120D2D08B9CC900591D99066
:10521000D1120D2D08B9C29E0591D990D1120D2D34
:1052200008B9040E151E0591D990D1120D2D08B99B
:10523000080E191E0591D990D1120D2D08B9A3950C
:10524000AF710591D990D1120D2D08B9A32BF001A2
:105250000591D990D1120D2D08B9CC900895F00187
:105260003296CC90C29E00C000C000C00591D9907B
:10527000D1120D2D08B9040E151E0591D990D11229
:105280000D2D08B9080E191E0591D990D1120D2DBA
:1052900008B9A395AF710591D990D1120D2D08B918
:1052A000A32BF0010591D990D1120D2D08B9CC9006
:1052B0000591D990D1120D2D08B9C29E0591D990B2
:1052C000D1120D2D08B9040E151E0591D990D112D9
:1052D0000D2D08B9080E191E0591D990D1120D2D6A
:1052E00008B9A395AF710591D990D1120D2D08B9C8
:1052F000A32BF0010591D990D1120D2D08B9CC90B6
:105300000591D990D1120D2D08B9C29E0591D99061
:10531000D1120D2D08B9040E151E0591D990D11288
:105320000D2D08B9080E191E0591D990D1120D2D19
:1053300008B9A395AF710591D990D1120D2D08B977
:10534000A32BF0010591D990D1120D2D08B9CC9065
:105350000591D990D1120D2D08B9C29E0591D99011
:10536000D1120D2D08B9040E151E0591D990D11238
:105370000D2D08B9080E191E0591D990D1120D2DC9
:1053800008B9A395AF710591D990D1120D2D08B927
:10539000A32BF0010591D990D1120D2D08B9CC9015
:1053A0000591D990D1120D2D08B9C29E0591D990C1
:1053B000D1120D2D08B9040E151E0591D990D112E8
:1053C0000D2D08B9080E191E0591D990D1120D2D79
:1053D00008B9A395AF710591D990D1120D2D08B9D7
:1053E000A32BF0010591D990D1120D2D08B9CC90C5
:1053F0000591D990D1120D2D08B9C29E0591D99071
:10540000D1120D2D08B9040E151E0591D990D11297
:105410000D2D08B9080E191E0591D990D1120D2D28
:1054200008B9A395AF710591D990D1120D2D08B986
:10543000A32BF0010591D990D1120D2D08B9CC9074
:105440000591D990D1120D2D08B9C29E0591D99020
:10545000D1120D2D08B9040E151E0591D990D11247
:105460000D2D08B9080E191E0591D990D1120D2DD8
:1054700008B9A395AF710591D990D1120D2D08B936
:10548000A32BF0010591D990D1120D2D08B9CC9024
:105490000591D990D1120D2D08B9C29E0591D990D0
:1054A000D1120D2D08B9040E151E0591D990D112F7
:1054B0000D2D08B9080E191E0591D990D1120D2D88
:1054C00008B9A395AF710591D990D1120D2D08B9E6
:1054D000A32BF0010591D990D1120D2D08B9CC90D4
:1054E0000591D990D1120D2D08B9C29E0591D99080
:1054F000D1120D2D08B9040E151E0591D990D112A7
:105500000D2D08B9080E191E0591D990D1120D2D37
:1055100008B9A395AF710591D990D1120D2D08B995
:10552000A32BF0010591D990D1120D2D08B9CC9083
:105530000591D990D1120D2D08B9C29E0591D9902F
:10554000D1120D2D08B9040E151E0591D990D11256
:105550000D2D08B9080E191E0591D990D1120D2DE7
:1055600008B9A395AF710591D990D1120D2D08B945
:10557000A32BF0010591D990D1120D2D08B9CC9033
:105580000591D990D1120D2D08B9C29E0591D990DF
:10559000D1120D2D08B9040E151E0591D990D11206
:1055A0000D2D08B9080E191E0591D990D1120D2D97
:1055B00008B9A395AF710591D990D1120D2D08B9F5
:1055C000A32BF0010591D990D1120D2D08B9CC90E3
:1055D0000591D990D1120D2D08B9C29E0591D9908F
:1055E000D1120D2D08B9040E151E0591D990D112B6
:1055F0000D2D08B9080E191E0591D990D1120D2D47
:1056000008B9A395AF710591D990D1120D2D08B9A4
:10561000A32BF0010591D990D1120D2D08B9CC9092
:105620000591D990D1120D2D08B9C29E0591D9903E
:10563000D1120D2D08B9040E151E0591D990D11265
:105640000D2D08B9080E191E0591D990D1120D2DF6
:1056500008B9A395AF710591D990D1120D2D08B954
:10566000A32BF0010591D990D1120D2D08B9CC9042
:105670000591D990D1120D2D08B9C29E0591D990EE
:10568000D1120D2D08B9040E151E0591D990D11215
:105690000D2D08B9080E191E0591D990D1120D2DA6
:1056A00008B9A395AF710591D990D1120D2D08B904
:1056B000A32BF0010591D990D1120D2D08B9CC90F2
:1056C0000591D990D1120D2D08B9C29E0591D9909E
:1056D000D1120D2D08B9040E151E0591D990D112C5
:1056E0000D2D08B9080E191E0591D990D1120D2D56
:1056F00008B9A395AF710591D990D1120D2D08B9B4
:10570000A32BF0010591D990D1120D2D08B9CC90A1
:105710000591D990D1120D2D08B9C29E0591D9904D
:10572000D1120D2D08B9040E151E0591D990D11274
:105730000D2D08B9080E191E0591D990D1120D2D05
:1057400008B9A395AF710591D990D1120D2D08B963
:10575000A32BF0010591D990D1120D2D08B9CC9051
:105760000591D990D1120D2D08B9C29E0591D990FD
:10577000D1120D2D08B9040E151E0591D990D11224
:105780000D2D08B9080E191E0591D990D1120D2DB5
:1057900008B9A395AF710591D990D1120D2D08B913
:1057A000A32BF0010591D990D1120D2D08B9CC9001
:1057B0000591D990D1120D2D08B9C29E0591D990AD
:1057C000D1120D2D08B9040E151E0591D990D112D4
:1057D0000D2D08B9080E191E0591D990D1120D2D65
:1057E00008B9A395AF710591D990D1120D2D08B9C3
:1057F000A32BF0010591D990D1120D2D08B9CC90B1
:105800000591D990D1120D2D08B9C29E0591D9905C
:10581000D1120D2D08B9040E151E0591D990D11283
:105820000D2D08B9080E191E0591D990D1120D2D14
:1058300008B9A395AF710591D990D1120D2D08B972
:10584000A32BF0010591D990D1120D2D08B9CC9060
:105850000591D990D1120D2D08B9C29E0591D9900C
:10586000D1120D2D08B9040E151E0591D990D11233
:105870000D2D08B9080E191E0591D990D1120D2DC4
:1058800008B9A395AF710591D990D1120D2D08B922
:10589000A32BF0010591D990D1120D2D08B9CC9010
:1058A0000591D990D1120D2D08B9C29E0591D990BC
:1058B000D1120D2D08B9040E151E0591D990D112E3
:1058C0000D2D08B9080E191E0591D990D1120D2D74
:1058D00008B9A395AF710591D990D1120D2D08B9D2
:1058E000A32BF0010591D990D1120D2D08B9CC90C0
:1058F0000591D990D1120D2D08B9C29E0591D9906C
:10590000D1120D2D08B9040E151E0591D990D11292
:105910000D2D08B9080E191E0591D990D1120D2D23
:1059200008B9A395AF710591D990D1120D2D08B981
:10593000A32BF0010591D990D1120D2D08B9CC906F
:105940000591D990D1120D2D08B9C29E0895F0018C
:105950003396CC90C29E040E151E00C000C0059167
:10596000D990D1120D2D08B9080E191E0591D990A4
:10597000D1120D2D08B9A395AF710591D990D1120F
:105980000D2D08B9A32BF0010591D990D1120D2D41
:1059900008B9CC900591D990D1120D2D08B9C29EAD
:1059A0000591D990D1120D2D08B9040E151E05913F
:1059B000D990D1120D2D08B9080E191E0591D99054
:1059C000D1120D2D08B9A395AF710591D990D112BF
:1059D0000D2D08B9A32BF0010591D990D1120D2DF1
:1059E00008B9CC900591D990D1120D2D08B9C29E5D
:1059F0000591D990D1120D2D08B9040E151E0591EF
:105A0000D990D1120D2D08B9080E191E0591D99003
:105A1000D1120D2D08B9A395AF710591D990D1126E
:105A20000D2D08B9A32BF0010591D990D1120D2DA0
:105A300008B9CC900591D990D1120D2D08B9C29E0C
:105A40000591D990D1120D2D08B9040E151E05919E
:105A5000D990D1120D2D08B9080E191E0591D990B3
:105A6000D1120D2D08B9A395AF710591D990D1121E
:105A70000D2D08B9A32BF0010591D990D1120D2D50
:105A800008B9CC900591D990D1120D2D08B9C29EBC
:105A90000591D990D1120D2D08B9040E151E05914E
:105AA000D990D1120D2D08B9080E191E0591D99063
:105AB000D1120D2D08B9A395AF710591D990D112CE
:105AC0000D2D08B9A32BF0010591D990D1120D2D00
:105AD00008B9CC900591D990D1120D2D08B9C29E6C
:105AE0000591D990D1120D2D08B9040E151E0591FE
:105AF000D990D1120D2D08B9080E191E0591D99013
:105B0000D1120D2D08B9A395AF710591D990D1127D
:105B10000D2D08B9A32BF0010591D990D1120D2DAF
:105B200008B9CC900591D990D1120D2D08B9C29E1B
:105B30000591D990D1120D2D08B9040E151E0591AD
:105B4000D990D1120D2D08B9080E191E0591D990C2
:105B5000D1120D2D08B9A395AF710591D990D1122D
:105B60000D2D08B9A32BF0010591D990D1120D2D5F
:105B700008B9CC900591D990D1120D2D08B9C29ECB
:105B80000591D990D1120D2D08B9040E151E05915D
:105B9000D990D1120D2D08B9080E191E0591D99072
:105BA000D1120D2D08B9A395AF710591D990D112DD
:105BB0000D2D08B9A32BF0010591D990D1120D2D0F
:105BC00008B9CC900591D990D1120D2D08B9C29E7B
:105BD0000591D990D1120D2D08B9040E151E05910D
:105BE000D990D1120D2D08B9080E191E0591D99022
:105BF000D1120D2D08B9A395AF710591D990D1128D
:105C00000D2D08B9A32BF0010591D990D1120D2DBE
:105C100008B9CC900591D990D1120D2D08B9C29E2A
:105C20000591D990D1120D2D08B9040E151E0591BC
:105C3000D990D1120D2D08B9080E191E0591D990D1
:105C4000D1120D2D08B9A395AF710591D990D1123C
:105C50000D2D08B9A32BF0010591D990D1120D2D6E
:105C600008B9CC900591D990D1120D2D08B9C29EDA
:105C70000591D990D1120D2D08B9040E151E05916C
:105C8000D990D1120D2D08B9080E191E0591D99081
:105C9000D1120D2D08B9A395AF710591D990D112EC
:105CA0000D2D08B9A32BF0010591D990D1120D2D1E
:105CB00008B9CC900591D990D1120D2D08B9C29E8A
:105CC0000591D990D1120D2D08B9040E151E05911C
:105CD000D990D1120D2D08B9080E191E0591D99031
:105CE000D1120D2D08B9A395AF710591D990D1129C
:105CF0000D2D08B9A32BF0010591D990D1120D2DCE
:105D000008B9CC900591D990D1120D2D08B9C29E39
:105D10000591D990D1120D2D08B9040E151E0591CB
:105D2000D990D1120D2D08B9080E191E0591D990E0
:105D3000D1120D2D08B9A395AF710591D990D1124B
:105D40000D2D08B9A32BF0010591D990D1120D2D7D
:105D500008B9CC900591D990D1120D2D08B9C29EE9
:105D60000591D990D1120D2D08B9040E151E05917B
:105D7000D990D1120D2D08B9080E191E0591D99090
:105D8000D1120D2D08B9A395AF710591D990D112FB
:105D90000D2D08B9A32BF0010591D990D1120D2D2D
:105DA00008B9CC900591D990D1120D2D08B9C29E99
:105DB0000591D990D1120D2D08B9040E151E05912B
:105DC000D990D1120D2D08B9080E191E0591D99040
:105DD000D1120D2D08B9A395AF710591D990D112AB
:105DE0000D2D08B9A32BF0010591D990D1120D2DDD
:105DF00008B9CC900591D990D1120D2D08B9C29E49
:105E00000591D990D1120D2D08B9040E151E0591DA
:105E1000D990D1120D2D08B9080E191E0591D990EF
:105E2000D1120D2D08B9A395AF710591D990D1125A
:105E30000D2D08B9A32BF0010591D990D1120D2D8C
:105E400008B9CC900591D990D1120D2D08B9C29EF8
:105E50000591D990D1120D2D08B9040E151E05918A
:105E6000D990D1120D2D08B9080E191E0591D9909F
:105E7000D1120D2D08B9A395AF710591D990D1120A
:105E80000D2D08B9A32BF0010591D990D1120D2D3C
:105E900008B9CC900591D990D1120D2D08B9C29EA8
:105EA0000591D990D1120D2D08B9040E151E05913A
:105EB000D990D1120D2D08B9080E191E0591D9904F
:105EC000D1120D2D08B9A395AF710591D990D112BA
:105ED0000D2D08B9A32BF0010591D990D1120D2DEC
:105EE00008B9CC900591D990D1120D2D08B9C29E58
:105EF0000591D990D1120D2D08B9040E151E0591EA
:105F0000D990D1120D2D08B9080E191E0591D990FE
:105F1000D1120D2D08B9A395AF710591D990D11269
:105F20000D2D08B9A32BF0010591D990D1120D2D9B
:105F300008B9CC900591D990D1120D2D08B9C29E07
:105F40000591D990D1120D2D08B9040E151E059199
:105F5000D990D1120D2D08B9080E191E0591D990AE
:105F6000D1120D2D08B9A395AF710591D990D11219
:105F70000D2D08B9A32BF0010591D990D1120D2D4B
:105F800008B9CC900591D990D1120D2D08B9C29EB7
:105F90000591D990D1120D2D08B9040E151E059149
:105FA000D990D1120D2D08B9080E191E0591D9905E
:105FB000D1120D2D08B9A395AF710591D990D112C9
:105FC0000D2D08B9A32BF0010591D990D1120D2DFB
:105FD00008B9CC900591D990D1120D2D08B9C29E67
:105FE0000591D990D1120D2D08B9040E151E0591F9
:105FF000D990D1120D2D08B9080E191E0591D9900E
:10600000D1120D2D08B9A395AF710591D990D11278
:106010000D2D08B9A32BF0010591D990D1120D2DAA
:1060200008B9CC900591D990D1120D2D08B9C29E16
:106030000591D990D1120D2D08B9040E151E0895A1
:10604000F0013496CC90C29E040E151E080E191E47
:1060500000C00591D990D1120D2D08B9A395AF714B
:106060000591D990D1120D2D08B9A32BF0010591FE
:10607000D990D1120D2D08B9CC900591D990D1129B
:106080000D2D08B9C29E0591D990D1120D2D08B9D8
:10609000040E151E0591D990D1120D2D08B9080EC8
:1060A000191E0591D990D1120D2D08B9A395AF7184
:1060B0000591D990D1120D2D08B9A32BF0010591AE
:1060C000D990D1120D2D08B9CC900591D990D1124B
:1060D0000D2D08B9C29E0591D990D1120D2D08B988
:1060E000040E151E0591D990D1120D2D08B9080E78
:1060F000191E0591D990D1120D2D08B9A395AF7134
:106100000591D990D1120D2D08B9A32BF00105915D
:10611000D990D1120D2D08B9CC900591D990D112FA
:106120000D2D08B9C29E0591D990D1120D2D08B937
:10613000040E151E0591D990D1120D2D08B9080E27
:10614000191E0591D990D1120D2D08B9A395AF71E3
:106150000591D990D1120D2D08B9A32BF00105910D
:10616000D990D1120D2D08B9CC900591D990D112AA
:106170000D2D08B9C29E0591D990D1120D2D08B9E7
:10618000040E151E0591D990D1120D2D08B9080ED7
:10619000191E0591D990D1120D2D08B9A395AF7193
:1061A0000591D990D1120D2D08B9A32BF0010591BD
:1061B000D990D1120D2D08B9CC900591D990D1125A
:1061C0000D2D08B9C29E0591D990D1120D2D08B997
:1061D000040E151E0591D990D1120D2D08B9080E87
:1061E000191E0591D990D1120D2D08B9A395AF7143
:1061F0000591D990D1120D2D08B9A32BF00105916D
:10620000D990D1120D2D08B9CC900591D990D11209
:106210000D2D08B9C29E0591D990D1120D2D08B946
:10622000040E151E0591D990D1120D2D08B9080E36
:10623000191E0591D990D1120D2D08B9A395AF71F2
:106240000591D990D1120D2D08B9A32BF00105911C
:10625000D990D1120D2D08B9CC900591D990D112B9
:106260000D2D08B9C29E0591D990D1120D2D08B9F6
:10627000040E151E0591D990D1120D2D08B9080EE6
:10628000191E0591D990D1120D2D08B9A395AF71A2
:106290000591D990D1120D2D08B9A32BF0010591CC
:1062A000D990D1120D2D08B9CC900591D990D11269
:1062B0000D2D08B9C29E0591D990D1120D2D08B9A6
:1062C000040E151E0591D990D1120D2D08B9080E96
:1062D000191E0591D990D1120D2D08B9A395AF7152
:1062E0000591D990D1120D2D08B9A32BF00105917C
:1062F000D990D1120D2D08B9CC900591D990D11219
:106300000D2D08B9C29E0591D990D1120D2D08B955
:10631000040E151E0591D990D1120D2D08B9080E45
:10632000191E0591D990D1120D2D08B9A395AF7101
:106330000591D990D1120D2D08B9A32BF00105912B
:10634000D990D1120D2D08B9CC900591D990D112C8
:106350000D2D08B9C29E0591D990D1120D2D08B905
:10636000040E151E0591D990D1120D2D08B9080EF5
:10637000191E0591D990D1120D2D08B9A395AF71B1
:106380000591D990D1120D2D08B9A32BF0010591DB
:10639000D990D1120D2D08B9CC900591D990D11278
:1063A0000D2D08B9C29E0591D990D1120D2D08B9B5
:1063B000040E151E0591D990D1120D2D08B9080EA5
:1063C000191E0591D990D1120D2D08B9A395AF7161
:1063D0000591D990D1120D2D08B9A32BF00105918B
:1063E000D990D1120D2D08B9CC900591D990D11228
:1063F0000D2D08B9C29E0591D990D1120D2D08B965
:10640000040E151E0591D990D1120D2D08B9080E54
:10641000191E0591D990D1120D2D08B9A395AF7110
:106420000591D990D1120D2D08B9A32BF00105913A
:10643000D990D1120D2D08B9CC900591D990D112D7
:106440000D2D08B9C29E0591D990D1120D2D08B914
:10645000040E151E0591D990D1120D2D08B9080E04
:10646000191E0591D990D1120D2D08B9A395AF71C0
:106470000591D990D1120D2D08B9A32BF0010591EA
:10648000D990D1120D2D08B9CC900591D990D11287
:106490000D2D08B9C29E0591D990D1120D2D08B9C4
:1064A000040E151E0591D990D1120D2D08B9080EB4
:1064B000191E0591D990D1120D2D08B9A395AF7170
:1064C0000591D990D1120D2D08B9A32BF00105919A
:1064D000D990D1120D2D08B9CC900591D990D11237
:1064E0000D2D08B9C29E0591D990D1120D2D08B974
:1064F000040E151E0591D990D1120D2D08B9080E64
:10650000191E0591D990D1120D2D08B9A395AF711F
:106510000591D990D1120D2D08B9A32BF001059149
:10652000D990D1120D2D08B9CC900591D990D112E6
:106530000D2D08B9C29E0591D990D1120D2D08B923
:10654000040E151E0591D990D1120D2D08B9080E13
:10655000191E0591D990D1120D2D08B9A395AF71CF
:106560000591D990D1120D2D08B9A32BF0010591F9
:10657000D990D1120D2D08B9CC900591D990D11296
:106580000D2D08B9C29E0591D990D1120D2D08B9D3
:10659000040E151E0591D990D1120D2D08B9080EC3
:1065A000191E0591D990D1120D2D08B9A395AF717F
:1065B0000591D990D1120D2D08B9A32BF0010591A9
:1065C000D990D1120D2D08B9CC900591D990D11246
:1065D0000D2D08B9C29E0591D990D1120D2D08B983
:1065E000040E151E0591D990D1120D2D08B9080E73
:1065F000191E0591D990D1120D2D08B9A395AF712F
:106600000591D990D1120D2D08B9A32BF001059158
:10661000D990D1120D2D08B9CC900591D990D112F5
:106620000D2D08B9C29E0591D990D1120D2D08B932
:10663000040E151E0591D990D1120D2D08B9080E22
:10664000191E0591D990D1120D2D08B9A395AF71DE
:106650000591D990D1120D2D08B9A32BF001059108
:10666000D990D1120D2D08B9CC900591D990D112A5
:106670000D2D08B9C29E0591D990D1120D2D08B9E2
:10668000040E151E0591D990D1120D2D08B9080ED2
:10669000191E0591D990D1120D2D08B9A395AF718E
:1066A0000591D990D1120D2D08B9A32BF0010591B8
:1066B000D990D1120D2D08B9CC900591D990D11255
:1066C0000D2D08B9C29E0591D990D1120D2D08B992
:1066D000040E151E0591D990D1120D2D08B9080E82
:1066E000191E0591D990D1120D2D08B9A395AF713E
:1066F0000591D990D1120D2D08B9A32BF001059168
:10670000D990D1120D2D08B9CC900591D990D11204
:106710000D2D08B9C29E0591D990D1120D2D08B941
:10672000040E151E0591D990D1120D2D08B9080E31
:10673000191E0895F0013596CC90C29E040E151EC8
:10674000080E191EA395AF710591D990D1120D2D88
:1067500008B9A32BF0010591D990D1120D2D08B9DC
:10676000CC900591D990D1120D2D08B9C29E0591FA
:10677000D990D1120D2D08B9040E151E0591D9908E
:10678000D1120D2D08B9080E191E0591D990D112FC
:106790000D2D08B9A395AF710591D990D1120D2D8A
:1067A00008B9A32BF0010591D990D1120D2D08B98C
:1067B000CC900591D990D1120D2D08B9C29E0591AA
:1067C000D990D1120D2D08B9040E151E0591D9903E
:1067D000D1120D2D08B9080E191E0591D990D112AC
:1067E0000D2D08B9A395AF710591D990D1120D2D3A
:1067F00008B9A32BF0010591D990D1120D2D08B93C
:10680000CC900591D990D1120D2D08B9C29E059159
:10681000D990D1120D2D08B9040E151E0591D990ED
:10682000D1120D2D08B9080E191E0591D990D1125B
:106830000D2D08B9A395AF710591D990D1120D2DE9
:1068400008B9A32BF0010591D990D1120D2D08B9EB
:10685000CC900591D990D1120D2D08B9C29E059109
:10686000D990D1120D2D08B9040E151E0591D9909D
:10687000D1120D2D08B9080E191E0591D990D1120B
:106880000D2D08B9A395AF710591D990D1120D2D99
:1068900008B9A32BF0010591D990D1120D2D08B99B
:1068A000CC900591D990D1120D2D08B9C29E0591B9
:1068B000D990D1120D2D08B9040E151E0591D9904D
:1068C000D1120D2D08B9080E191E0591D990D112BB
:1068D0000D2D08B9A395AF710591D990D1120D2D49
:1068E00008B9A32BF0010591D990D1120D2D08B94B
:1068F000CC900591D990D1120D2D08B9C29E059169
:10690000D990D1120D2D08B9040E151E0591D990FC
:10691000D1120D2D08B9080E191E0591D990D1126A
:106920000D2D08B9A395AF710591D990D1120D2DF8
:1069300008B9A32BF0010591D990D1120D2D08B9FA
:10694000CC900591D990D1120D2D08B9C29E059118
:10695000D990D1120D2D08B9040E151E0591D990AC
:10696000D1120D2D08B9080E191E0591D990D1121A
:106970000D2D08B9A395AF710591D990D1120D2DA8
:1069800008B9A32BF0010591D990D1120D2D08B9AA
:10699000CC900591D990D1120D2D08B9C29E0591C8
:1069A000D990D1120D2D08B9040E151E0591D9905C
:1069B000D1120D2D08B9080E191E0591D990D112CA
:1069C0000D2D08B9A395AF710591D990D1120D2D58
:1069D00008B9A32BF0010591D990D1120D2D08B95A
:1069E000CC900591D990D1120D2D08B9C29E059178
:1069F000D990D1120D2D08B9040E151E0591D9900C
:106A0000D1120D2D08B9080E191E0591D990D11279
:106A10000D2D08B9A395AF710591D990D1120D2D07
:106A200008B9A32BF0010591D990D1120D2D08B909
:106A3000CC900591D990D1120D2D08B9C29E059127
:106A4000D990D1120D2D08B9040E151E0591D990BB
:106A5000D1120D2D08B9080E191E0591D990D11229
:106A60000D2D08B9A395AF710591D990D1120D2DB7
:106A700008B9A32BF0010591D990D1120D2D08B9B9
:106A8000CC900591D990D1120D2D08B9C29E0591D7
:106A9000D990D1120D2D08B9040E151E0591D9906B
:106AA000D1120D2D08B9080E191E0591D990D112D9
:106AB0000D2D08B9A395AF710591D990D1120D2D67
:106AC00008B9A32BF0010591D990D1120D2D08B969
:106AD000CC900591D990D1120D2D08B9C29E059187
:106AE000D990D1120D2D08B9040E151E0591D9901B
:106AF000D1120D2D08B9080E191E0591D990D11289
:106B00000D2D08B9A395AF710591D990D1120D2D16
:106B100008B9A32BF0010591D990D1120D2D08B918
:106B2000CC900591D990D1120D2D08B9C29E059136
:106B3000D990D1120D2D08B9040E151E0591D990CA
:106B4000D1120D2D08B9080E191E0591D990D11238
:106B50000D2D08B9A395AF710591D990D1120D2DC6
:106B600008B9A32BF0010591D990D1120D2D08B9C8
:106B7000CC900591D990D1120D2D08B9C29E0591E6
:106B8000D990D1120D2D08B9040E151E0591D9907A
:106B9000D1120D2D08B9080E191E0591D990D112E8
:106BA0000D2D08B9A395AF710591D990D1120D2D76
:106BB00008B9A32BF0010591D990D1120D2D08B978
:106BC000CC900591D990D1120D2D08B9C29E059196
:106BD000D990D1120D2D08B9040E151E0591D9902A
:106BE000D1120D2D08B9080E191E0591D990D11298
:106BF0000D2D08B9A395AF710591D990D1120D2D26
:106C000008B9A32BF0010591D990D1120D2D08B927
:106C1000CC900591D990D1120D2D08B9C29E059145
:106C2000D990D1120D2D08B9040E151E0591D990D9
:106C3000D1120D2D08B9080E191E0591D990D11247
:106C40000D2D08B9A395AF710591D990D1120D2DD5
:106C500008B9A32BF0010591D990D1120D2D08B9D7
:106C6000CC900591D990D1120D2D08B9C29E0591F5
:106C7000D990D1120D2D08B9040E151E0591D99089
:106C8000D1120D2D08B9080E191E0591D990D112F7
:106C90000D2D08B9A395AF710591D990D1120D2D85
:106CA00008B9A32BF0010591D990D1120D2D08B987
:106CB000CC900591D990D1120D2D08B9C29E0591A5
:106CC000D990D1120D2D08B9040E151E0591D99039
:106CD000D1120D2D08B9080E191E0591D990D112A7
:106CE0000D2D08B9A395AF710591D990D1120D2D35
:106CF00008B9A32BF0010591D990D1120D2D08B937
:106D0000CC900591D990D1120D2D08B9C29E059154
:106D1000D990D1120D2D08B9040E151E0591D990E8
:106D2000D1120D2D08B9080E191E0591D990D11256
:106D30000D2D08B9A395AF710591D990D1120D2DE4
:106D400008B9A32BF0010591D990D1120D2D08B9E6
:106D5000CC900591D990D1120D2D08B9C29E059104
:106D6000D990D1120D2D08B9040E151E0591D99098
:106D7000D1120D2D08B9080E191E0591D990D11206
:106D80000D2D08B9A395AF710591D990D1120D2D94
:106D900008B9A32BF0010591D990D1120D2D08B996
:106DA000CC900591D990D1120D2D08B9C29E0591B4
:106DB000D990D1120D2D08B9040E151E0591D99048
:106DC000D1120D2D08B9080E191E0591D990D112B6
:106DD0000D2D08B9A395AF710591D990D1120D2D44
:106DE00008B9A32BF0010591D990D1120D2D08B946
:106DF000CC900591D990D1120D2D08B9C29E059164
:106E0000D990D1120D2D08B9040E151E0591D990F7
:106E1000D1120D2D08B9080E191E0591D990D11265
:106E20000D2D08B9A395AF71089528980E94A2412D
:106E3000E7E1EA95F1F7289AE3D0E0E0F6E0C6D082
:106E4000E0FF05D0E0FF02C00E94C7400895EF9325
:106E5000E091980AE53EE0F5E531D0F12F923F92BE
:106E60004F925F926F927F928F929F92AF92BF925A
:106E7000CF92DF92EF92FF920F931F932F933F9346
:106E80004F935F936F937F938F939F93AF93BF9332
:106E9000CF93DF930E94CE20DF91CF91BF91AF912E
:106EA0009F918F917F916F915F914F913F912F9122
:106EB0001F910F91FF90EF90DF90CF90BF90AF9018
:106EC0009F908F907F906F905F904F903F902F900A
:106ED000EF910895FF93EF93EFB7EF93E091840064
:106EE000EE50E13000F0E23000F0E33000F0E4304A
:106EF00000F0E53000F0E63000F0E73000F0E83078
:106F000000F0E93000F005D0EF91EFBFEF91FF9175
:106F100018950F921F92E4E9F1E40090970A000C93
:106F20001124E00DF11D05901490F00109951F90BA
:106F30000F90089528980E94A241E5E1EA95F1F7A3
:106F4000E091980AEA95E093980A289A00000000D8
:106F5000089528980E94CB41289A0000E1E0F6E0CD
:106F600035D047D0089528980E94CB41E0EB00002F
:106F7000EA95E9F700000000289AF6E0E2E026D062
:106F8000089528980E94CB41289A0000E3E0FDEF85
:106F90001DD0E091980AE53091F4E0919A0AE13031
:106FA0000000F091A80A19F4F091A80AF195E3E025
:106FB000E0938900EDE8EF0FE09388000895E3E0A7
:106FC000E0938900EDE8E093880008950090980A26
:106FD0000A9410905F0011FC0F2E0092980A009006
:106FE000970A11FC0E2E0092970AE0E011FCE1E0F6
:106FF0000895E3E0E0938900EDE8E09388000895C8
:10700000E7E0E0938900EBE1E09388000895E0E495
:10701000F4E0A0ECB1E060E06D933197E9F7112462
:107020000895CC03CC03CC03CC03CC03CC03CC031A
:10703000CC03CC03CC03CC03CC03CC03CC03CC03D8
:10704000CC03CC03CC03CC03CC03CC03CC03CC03C8
:10705000CC03CC03CC03CC03CC03CC03CC03CC03B8
:10706000CC03CC03CC03CC03CC03CC03CC03CC03A8
:10707000CC03CC03CC03CC03CC03CC03CC03CC0398
:10708000CC03CC03CC039927772720E2629F080E1C
:10709000191EA0ECB1E0A00DB11D4C931124089570
:1070A0000895992720E2629F080E191EA0ECB1E016
:1070B000A00DB11D50919F0A450F4C9311240895C6
:1070C00080939F0A089580937F0690938006089589
:1070D00080937E060895EF92FF920F931F93CF93B4
:1070E000DF93E0E6F6E020E0822F60814181EF93BC
:1070F000FF932F930E9480472F91FF91EF913F962E
:107100002395223088F3552722E0662775E081E831
:1071100096E0E0E6F6E030854281EC01579FC00D35
:10712000D11D540F442349F0317039F069936993AC
:107130006993699369934A95C9F73F962A9559F7D8
:1071400031E020917E06213011F43091960A00E062
:1071500016E0780123E0A5E0B0E241E0F701329FBC
:10716000E00DF11D008111811030E9F1183DD8F5D5
:107170000030C9F10A38B8F560E0712F760F783029
:1071800068F1783D58F57850EC017A9FC00DD11D1B
:107190000880002021F46B9F030E08821FC0098025
:1071A000002021F46B9F030E098218C00A80002082
:1071B00021F46B9F030E0A8211C00B80002021F482
:1071C0006B9F030E0B820AC00C80002039F46B9F6A
:1071D000030E0C82032E0A940092960A259673954C
:1071E0006395683050F23395303208F031E04395C2
:1071F000403208F4B3CF7091960A703208F071E013
:107200007093960A552722E0662775E0E0E6F6E0DF
:1072100030854281EC01579FC00DD11D540F44238E
:1072200049F0317039F4699369936993699369936B
:107230004A95C9F73F962A9559F71124DF91CF91C6
:107240001F910F91FF90EF90089580939D0A909366
:107250009E0A08958091990A089511241092990A1E
:10726000089580E891E08093610090936100089513
:1072700080E890E08093610090936100089580938E
:10728000A80A0895882329F48091A00A9091A10A60
:1072900008958091A40A9091A50A0895882329F45D
:1072A0008091A20A9091A30A08958091A60A9091D4
:1072B000A70A089578E07A95F1F700000197D1F7D1
:1072C0000895F999FECF92BD81BD60BDF894FA9AF8
:1072D000F99A78940895F999FECF92BD81BDF894FA
:1072E000F89A80B57894089528E088E190E00FB688
:1072F000F894A895809360000FBE20936000FFCFA4
:1073000081E08093FD0C08951F9380E090E00E943F
:107310006B39182F81E090E00E946B3990E0382F94
:1073200020E0210F311D2A55354509F491E0892FC0
:107330001F910895BF92CF92DF92EF92FF920F9329
:107340001F93CF93DF936C01062FB72E0E948439D1
:107350008823F1F18FEFC8168FEFD80611F481E082
:107360003AC0EE24FF24C7010E946B39182FC701D1
:1073700001960E946B39D82FC0E0CE01810F911D7C
:107380008C159D0521F4E114F10459F423C080E229
:1073900090E0E80EF91E90E0E91694E0F90619F77E
:1073A00019C0802F9B2D9C01E90180E2C82ED12CB1
:1073B000C20ED31E87010F5F1F4FC7010E946B399A
:1073C0008993CC15DD0511F480E005C07801F2CF7A
:1073D00084E001C083E0DF91CF911F910F91FF9076
:1073E000EF90DF90CF90BF900895BF92CF92DF9241
:1073F000EF92FF920F931F93CF93DF936C010E9444
:107400008439882311F484E04EC0F6018081918193
:10741000FFEF8F3F9F0709F445C08A55954509F452
:1074200041C002E010E020E4E22EF12CC7010E94EE
:107430006B39B82EC70101960E946B39D82FC0E076
:107440009E012B0D311DF60180819181281739078E
:1074500019F41123B1F00EC02F5F3F4F19F411231F
:1074600009F4102F0F5F80E290E0E80EF91E00345F
:10747000E9F623C0E12EFF2495E0EE0CFF1C9A955F
:10748000E1F7C0E0D0E0F601EC0FFD1FCE018E0D5C
:107490009F1D60810E9461392196C032D10599F704
:1074A00080E001C081E0DF91CF911F910F91FF90AB
:1074B000EF90DF90CF90BF9008951123D9F682E02E
:1074C000F2CFFF920F931F93CF93DF93129A809185
:1074D000FD0C882329F081E090E00E945A3902C017
:1074E000C895C895129800E010E0C0E0D0E0FF24F5
:1074F00016950795D695C79513988091FD0C88230E
:1075000029F085E090E00E945A3902C0C895C895DC
:10751000009B1068019BD068139A8091FD0C882312
:1075200029F085E090E00E945A3902C0C895C895BC
:10753000F39480E1F816E1F61093A10A0093A00AF3
:10754000D093A50AC093A40ADF91CF911F910F9108
:10755000FF9008958091FD0C8823E1F00E94613A2C
:107560008091A00A9091A10A97FF05C08091A00A7E
:107570009091A10A0AC08091A40A9091A50A97FF50
:1075800009C08091A40A9091A50A892F86958695B5
:10759000837008958FEF0895FF920F931F93F82E35
:1075A0008091FD0C882309F428C006E00E94AA3AC5
:1075B0008F1511F481E022C088EE93E00E945A39C1
:1075C00010E0129A1398C895C895C895C895C895A3
:1075D000C895C895139A129882E090E00E945A3993
:1075E000C895C895C895C895C895C895C8951F5F92
:1075F0001F3139F70F5F09F0D9CF80E01F910F914C
:10760000FF900895FF920F931F93CF93DF930E94F3
:10761000613A8091A00A9091A10A97FD06C08091DD
:10762000A40A9091A50A97FF27C081E090E00E94EC
:107630005A3900E010E0C0E0D0E0FF24000F111F35
:10764000CC0FDD1F1398C895C895C895C895009BA9
:107650000160019BC160139A88E090E00E945A3952
:10766000F39480E1F81651F71093A30A0093A20A4D
:10767000D093A70AC093A60ADF91CF911F910F91D3
:10768000FF9008950F931F9303E318E0C8010E9431
:10769000E13B80E790E090936606809365060E9448
:1076A00007388FE090E00E949D48C8010E94E13BAE
:1076B00080E06FEF41E00E947D3F00EC17E088E042
:1076C0006CE0A8010E94444A83E090E00E949D483B
:1076D00088E06CE044EF57E00E94444A82E090E08A
:1076E0000E949D4888E06CE0A8010E94444A84E121
:1076F00090E00E949D4880E590E00E949D480E9495
:10770000073884E190E00E949D481F910F910895F1
:1077100090E026E130E0829FF001839FF00D929F80
:10772000F00D1124E050F34F628708956093F10C3F
:10773000089590E026E130E0829FF001839FF00DF4
:10774000929FF00D1124E050F34F1386118208959B
:1077500090E026E130E0829FF001839FF00D929F40
:10776000F00D1124E050F34F81E0838B089590E0F9
:1077700026E130E0829FF001839FF00D929FF00D93
:107780001124E050F34F6187089590E026E130E046
:10779000829FF001839FF00D929FF00D1124E05025
:1077A000F34F6483089590E026E130E0829FF0017A
:1077B000839FF00D929FF00D1124E050F34F6583ED
:1077C000089590935B0D80935A0D8FE68093600D22
:1077D0001092C00AE0E0FDE021E08FEF98E1208305
:1077E00010868683878314861182958376963DE082
:1077F000E835F307A1F708951092010D1092170DC7
:1078000010922D0D1092430D01969093640D80936C
:10781000630D9093FF0C8093FE0C9093670D809303
:10782000660D1092620D1092610D1092590D10921A
:10783000580D10925C0D81E08093C00A10925F0D8C
:1078400010925E0D08958091FE0C9091FF0C0E94A5
:10785000FC3B089580910A0D87FD03C08AEF809359
:107860000A0D8091200D87FD03C08AEF8093200DC3
:107870008091360D87FD03C08AEF8093360D80918D
:107880004C0D87FD03C08AEF80934C0D1092C00A07
:10789000089581E08093C00A0895DC01ED91FC9188
:1078A0001197AF014F5F5F4F11965C934E93E49138
:1078B0002E2F30E0E7FF13C02F7730703695322F30
:1078C000222737952795FA014F5F5F4FE4918E2F5E
:1078D0008F77280F311DE7FDF1CF4D935C93C901E0
:1078E00008958093600D08950E949F400895EF923F
:1078F000FF920F931F93CF93DF93182F062FF42E31
:10790000E22EC82FD0E086E190E0C89FF001C99F29
:10791000F00DD89FF00D1124E050F34F838588239C
:1079200021F08181882309F088C0EE2091F486E15E
:1079300090E0C89FF001C99FF00DD89FF00D112471
:10794000E050F34F138A8285882309F076C01086B1
:1079500074C0133059F481E091E09093F30C80935C
:10796000F20C81E08093F10C0F2D08C0812F60E0B4
:107970000E949F40812F6F2D0E9480400F3799F405
:1079800086E190E0C89FF001C99FF00DD89FF00DEF
:107990001124E050F34F80915D0D87878EE59DE0C7
:1079A000958B848B30C089E0089FC0011124E09141
:1079B0005A0DF0915B0DE80FF91F339645915491E4
:1079C0004115510571F486E190E0C89FF001C99F0F
:1079D000F00DD89FF00D1124E050F34F158A148A52
:1079E00012C0FA01249186E190E0C89FF001C99F7E
:1079F000F00DD89FF00D1124E050F34F27874F5F13
:107A00005F4F558B448B86E190E0C89FF001C99F82
:107A1000F00DD89FF00D1124E050F34F108A12861C
:107A2000048711829FEF9187E086F282118A81E0BC
:107A30008387138A128A14829683DF91CF911F91D4
:107A40000F91FF90EF900895CF92DF92FF920F93E6
:107A50001F93CF93DF93E9E0FDE08181282F332747
:107A600027FD30958081280F311D2F3F310519F0FA
:107A700014F02FEF30E0C90137FF02C080E090E042
:107A8000808376964DE0E136F40739F78091C00A9D
:107A9000882309F028C144C1E091630DF091640D81
:107AA0009F012F5F3F4F3093640D2093630D4491EE
:107AB0004F3F69F5A9014F5F5F4F5093640D4093AD
:107AC000630DF90184918F3219F41092C00A19C123
:107AD000863009F0FBC0FA013196CF0101969093F0
:107AE000640D8093630DE491E33529F49093670D61
:107AF0008093660DEBC0E53409F0E8C08091660D17
:107B00009091670D9093640D8093630DDFC047FFE4
:107B100002C040935C0D542F5F70842F90E0807FF3
:107B20009070803B910531F1803C910581F1803965
:107B3000910509F043C0C9010196F90144910196EC
:107B40009093640D8093630D0197FC012491852F20
:107B500090E08C9FF0018D9FF00D9C9FF00D112403
:107B6000E050F34F8081882309F4B0C0220F852FA5
:107B7000648553C0C9010196F9014491019690931F
:107B8000640D8093630D0197FC01249153C02F5F16
:107B90003F4F3093640D2093630D21503040F90125
:107BA0002491852F90E08C9FF0018D9FF00D9C9F7C
:107BB000F00D1124E050F34F248788C080915C0DB4
:107BC000582F5F7090E0807F9070803B910541F16D
:107BD000803C910509F46EC08039910509F076C0AA
:107BE0002F5F3F4F3093640D2093630D2150304041
:107BF000F9012491852F90E08C9FD0018D9FB00DCD
:107C00009C9FB00D1124A050B34F8C91882309F490
:107C10005DC0220F852F1C966C910E94773C56C048
:107C20002F5F3F4F3093640D2093630D2150304000
:107C3000F9012491473071F4852F90E08C9FF00179
:107C40008D9FF00D9C9FF00D1124E050F34F220FFB
:107C500027833CC04B3071F4852F90E08C9FF0015E
:107C60008D9FF00D9C9FF00D1124E050F34F220FDB
:107C700026832CC04C3571F4852F90E08C9FF00149
:107C80008D9FF00D9C9FF00D1124E050F34F220FBB
:107C900024831CC04436D1F4852F90E08C9FF001E2
:107CA0008D9FF00D9C9FF00D1124E050F34F220F9B
:107CB00025830CC0852F90E08C9FF0018D9FF00DE7
:107CC0009C9FF00D1124E050F34F448783E69DE024
:107CD0000E944D3C9093620D8093610D1092590D5E
:107CE0001092580D02C0C6E1D0E06091580D70911D
:107CF000590D8091610D9091620D6817790709F413
:107D0000CBCE6F5F7F4F7093590D6093580D80916C
:107D10005E0D90915F0D019690935F0D80935E0DC7
:107D200002ED1CE0C1E0DDE0FF24BFEFCB2ED12C43
:107D30008A89882309F05EC08B899C89892B09F484
:107D400056C09F858E85981708F04CC050C08B8513
:107D50002B893C898F37E9F4D9018D91BC8BAB8B92
:107D60008F3F01F1F90161811196BC8BAB8BE82F3C
:107D7000F0E0EE0FFF1FE45CF74F0190F081E02D83
:107D80008F2D0995EB89FC8981918E87FC8BEB8B7C
:107D900028C0A9014F5F5F4F5C8B4B8BF901849129
:107DA0008F3F21F418821C8A1B8A21C04F5F5F4FCE
:107DB0005C8B4B8B41505040FA01649190E0880FEE
:107DC000991F845C974FFC01259134918F2DF90107
:107DD0000995EB89FC893196FC8BEB8B3197E4910B
:107DE000EE871F869F858E85981709F4B0CF8F8503
:107DF0008F5F8F878A85882319F420E030E06BC07D
:107E000088898F3F11F08F5F888B9F81992309F4B8
:107E10005CC02885222309F458C08E81882309F488
:107E200054C04091600D442309F44FC0899FC001A4
:107E3000112480509F4F892F992730E0B901869FE8
:107E40009001879F300D969F300D112420503F4F99
:107E5000232F33278D8190E0FC012E9FC0012F9F9F
:107E6000900D3E9F900D112480509F4F892F992790
:107E7000242F30E0AC01429FC001439F900D529FE0
:107E8000900D112480509F4F292F33278B818823F9
:107E9000F1F0EA81F0E0E050FC47E491E058E89F1F
:107EA000C001112480509F4F892F9927B601681B6C
:107EB000790B629FC001639F900D729F900D1124FA
:107EC00080509F4F292F332702C020E030E08A8165
:107ED0009C81890F8A83F8012083F394065F1F4FEA
:107EE0006696F4E0FF1609F023CFDF91CF911F9142
:107EF0000F91FF90DF90CF9008951F93CF93DF9362
:107F0000582F89E0589FC001112420915A0D3091BB
:107F10005B0D280F391FC9010396FC01A591B4918F
:107F2000F90184918150823010F413E01DC08091DA
:107F3000170D8823B1F08091230D851711F4442388
:107F400081F480912D0D882371F08091390D851772
:107F500011F4442341F49091270D80913D0D891730
:107F600010F411E001C012E0212F30E0FD01449136
:107F700086E190E0289FE001299FD00D389FD00D29
:107F80001124C050D34F4F871196BD8BAC8B188AEC
:107F900080E58A8368878FEF89871A861B8A198A0A
:107FA00021E02B871A8A5D8729831C828E831330F8
:107FB00049F481E091E09093F30C8093F20C2093CC
:107FC000F10C08C0812F60E50E948040812F6A89F2
:107FD0000E949F40DF91CF911F910895FF920F93D0
:107FE0001F93082FF62E0E94804010E086E190E05B
:107FF000089FF001099FF00D189FF00D1124E0502B
:10800000F34FF2821F910F91FF900895962F482F02
:1080100050E026E130E0429FF001439FF00D529F77
:10802000F00D1124E050F34F6281691B62830E94BE
:1080300080400895482F50E026E130E0429FF00153
:10804000439FF00D529FF00D1124E050F34F9281A9
:10805000690F62830E9480400895000000000000C4
:108060000000000000000000000000000000000010
:108070000000000000000000000000000000000000
:1080800000000000000000000000000000000000F0
:1080900000000000000000000000000000000000E0
:1080A00000000000000000000000000000000000D0
:1080B00000000000000000000000000000000000C0
:1080C00000000000000000000000000000000000B0
:1080D00000000000000000000000000000000000A0
:1080E0000000000000000000000000000000000090
:1080F0000000000000000000000000000000000080
:1081000099277727833008F00895E0E0FEE8660FAE
:10811000771FE60FF71FA591B491E2EDFCE02AE08E
:10812000289FE00DF11DA183B28311240895909141
:10813000F10C9170880F892B8093F10C0895992789
:108140007727E2EDFCE02AE0289FE00DF11D6E3F6D
:1081500031F46091F10C6E7F6093F10C0BC06F3FB6
:1081600031F46091F10C6E6F6093F10C03C074E810
:10817000760F75831124089599277727E2EDFCE0A7
:108180002AE0289FE00DF11D6083112408952F93AC
:108190003F934F935F936F937F938F939F93AF938F
:1081A000BF93789411240E9479480E946B380E94F2
:1081B000023B0E94243D2F923F924F925F926F921A
:1081C0007F928F929F92AF92BF92CF92DF92EF9267
:1081D000FF920F931F93CF93DF930090CF0C00205B
:1081E00019F4A1ECBAE002C0A7ECBBE001E0002664
:1081F0000092CF0C02E00093D00C5091F00C6091F3
:10820000F20C7091F30C8091F40C2090D30C309010
:10821000D40C4090D60C5090D70C6090D50C109197
:10822000D20C7090DD0C8090DE0C9090DF0CA09052
:10823000E00CB090E10C2091DC0CC090E70CD090E9
:10824000E80CE090EA0CF090EB0C0091E90C309116
:10825000E60C9FEF620C431CF201449141030024A1
:108260000008C12DD02D970CA81CF50144914203A4
:1082700000240008C10DD01D0C0DED1CF701449128
:10828000430300240008C10DD01D8A956AF4409173
:10829000F10C842F8695062E0694062600FA769514
:1082A000679576F940FF66F940E860FD4FE74503C2
:1082B00000240008C10DD01D0024C038D0050CF0EA
:1082C000CFE70A94C038D0050CF4C0E8C058CD936D
:1082D0009A9509F0BFCF4091D00C4A954093D00CAD
:1082E00097E009F0B7CF6092D50C4092D60C9092EF
:1082F000DF0CA092E00C0093E90CE092EA0C609392
:10830000F20C7093F30C8093F40CDF91CF911F91DA
:108310000F91FF90EF90DF90CF90BF90AF909F9024
:108320008F907F906F905F904F903F902F90BF9174
:10833000AF919F918F917F916F915F914F913F91FD
:108340002F9108950C94A4410C94A6410F931F9370
:108350002ABDE091CD0CF091CE0C0191000000936C
:10836000B3000CE0ED3CF00710F40000000010F04A
:10837000E1ECFAE0E093CD0CF093CE0CC895C895F3
:10838000C895C895C895C8950000000000002AB59A
:108390001F910F9108950000E091980AE0FFD6CF59
:1083A000E1E1EA95F1F70000000008950000000007
:1083B00000000000000000000000000000000000BD
:1083C00000000000000000000000000000000000AD
:1083D000000000000000000000000000000000009D
:1083E000000000000000000000000000000000008D
:1083F000000000000000000000000000000000007D
:10840000000306090C101316191C1F2225282B2EF9
:10841000313336393C3F414447494C4E515355580E
:108420005A5C5E60626466686A6B6D6F70717374CB
:10843000757678797A7A7B7C7D7D7E7E7E7F7F7F84
:108440007F7F7F7F7E7E7E7D7D7C7B7A7A7978766A
:1084500075747371706F6D6B6A68666462605E5C80
:108460005A585553514E4C494744413F3C39363395
:10847000312E2B2825221F1C191613100C09060358
:1084800000FDFAF7F4F0EDEAE7E4E1DEDBD8D5D25F
:10849000CFCDCAC7C4C1BFBCB9B7B4B2AFADABA82A
:1084A000A6A4A2A09E9C9A9896959391908F8D8C4D
:1084B0008B8A888786868584838382828281818174
:1084C0008181818182828283838485868687888A6E
:1084D0008B8C8D8F9091939596989A9C9EA0A2A438
:1084E000A6A8ABADAFB2B4B7B9BCBFC1C4C7CACD03
:1084F000CFD2D5D8DBDEE1E4E7EAEDF0F4F7FAFD20
:10850000808182838485868788898A8B8C8D8E8FF3
:10851000909192939495969798999A9B9C9D9E9FE3
:10852000A0A1A2A3A4A5A6A7A8A9AAABACADAEAFD3
:10853000B0B1B2B3B4B5B6B7B8B9BABBBCBDBEBFC3
:10854000C0C1C2C3C4C5C6C7C8C9CACBCCCDCECFB3
:10855000D0D1D2D3D4D5D6D7D8D9DADBDCDDDEDFA3
:10856000E0E1E2E3E4E5E6E7E8E9EAEBECEDEEEF93
:10857000F0F1F2F3F4F5F6F7F8F9FAFBFCFDFEFF83
:10858000000102030405060708090A0B0C0D0E0F73
:10859000101112131415161718191A1B1C1D1E1F63
:1085A000202122232425262728292A2B2C2D2E2F53
:1085B000303132333435363738393A3B3C3D3E3F43
:1085C000404142434445464748494A4B4C4D4E4F33
:1085D000505152535455565758595A5B5C5D5E5F23
:1085E000606162636465666768696A6B6C6D6E6F13
:1085F000707172737475767778797A7B7C7D7E7F03
:1086000000020406080A0C0E10121416181A1C1E7A
:1086100020222426282A2C2E30323436383A3C3E6A
:1086200040424446484A4C4E50525456585A5C5E5A
:1086300060626466686A6C6E70727476787A7C7E4A
:108640007F7D7B79777573716F6D6B69676563612A
:108650005F5D5B59575553514F4D4B49474543411A
:108660003F3D3B39373533312F2D2B29272523210A
:108670001F1D1B19171513110F0D0B0907050301FA
:10868000FFFDFBF9F7F5F3F1EFEDEBE9E7E5E3E1EA
:10869000DFDDDBD9D7D5D3D1CFCDCBC9C7C5C3C1DA
:1086A000BFBDBBB9B7B5B3B1AFADABA9A7A5A3A1CA
:1086B0009F9D9B99979593918F8D8B8987858381BA
:1086C00080828486888A8C8E90929496989A9C9EBA
:1086D000A0A2A4A6A8AAACAEB0B2B4B6B8BABCBEAA
:1086E000C0C2C4C6C8CACCCED0D2D4D6D8DADCDE9A
:1086F000E0E2E4E6E8EAECEEF0F2F4F6F8FAFCFE8A
:108700007F7F7F7F7F7F7F7F7F7F7F7F7F7F7F7F79
:108710007F7F7F7F7F7F7F7F7F7F7F7F7F7F7F7F69
:108720007F7F7F7F7F7F7F7F7F7F7F7F7F7F7F7F59
:108730007F7F7F7F7F7F7F7F7F7F7F7F7F7F7F7F49
:108A00000309131E28313A40464C5054585B5E61AE
:108A1000636567696B6C6E6F70717273747576776E
:108A2000777879797A7A7B7B7C7C7C7D7D7D7E7E94
:108A30007E7E7F7F7F7F7F7F7F7F7F7F7F7F7F7F48
:108A40007F7F7F7F7F7F7F7F7F7F7F7F7F7E7E7E39
:108A50007E7D7D7D7C7C7C7B7B7A7A79797877776B
:108A6000767574737271706F6E6C6B696765636134
:108A70005E5B5854504C46403A31281E130903009F
:108A8000C6CCD5DBDFE3E5E7E9EAEBECEDEEEFEFB3
:108A9000F0F0F0F1F1F1F1F2F2F2F2F2F2F2F2F3BF
:108AA000F3F3F3F3F3F3F3F3F3F3F3F3F3F3F3F396
:108AB000F3F3F3F3F3F3F3F3F3F3F3F3F3F3F3F386
:108AC000F3F3F3F3F3F3F3F3F3F3F3F3F3F3F3F376
:108AD000F3F3F3F3F3F3F3F3F3F3F3F3F3F3F3F366
:108AE000F2F2F2F2F2F2F2F2F1F1F1F1F0F0F0EF73
:108AF000EFEEEDECEBEAE9E7E5E3DFDBD5CCC60032
:108B000000283D42302D2C2B2C2D2E2F303233358A
:108B100037393B3D3F414345484A4C4E50535557EA
:108B2000595B5D5F61636567696B6C6E70717374CF
:108B3000757778797A7B7C7D7D7E7E7F7F7F7F7F76
:108B40007F7F7F7F7F7F7E7E7D7D7C7B7A7978775C
:108B500075747371706E6C6B69676563615F5D5B83
:108B600059575553504E4C4A484543413F3D3B3978
:108B700037353332302F2E2D2C2B2C2D30423D28E3
:108B800000E9E5FED4D7D7D7D6D4D2D0CECCCAC848
:108B9000C6C3C1BFBDBAB8B6B4B1AFADABA9A7A586
:108BA000A3A19F9E9C9A999795949391908F8D8C59
:108BB0008B8A898888878685858484848383838358
:108BC0008383838383848484858586878888898A50
:108BD0008B8C8D8F909193949597999A9C9E9FA141
:108BE000A3A5A7A9ABADAFB1B4B6B8BABDBFC1C359
:108BF000C6C8CACCCED0D2D4D6D7D7D7D4FEE5E912
:108C0000F9F8F9F5EBE1DDDEE0E2E4E5E6E5E4E2E2
:108C1000DED9D2CAC1B7ACA299918A8683818080FD
:108C20008182838586888A8C8D8F90929395969782
:108C300098999A9B9B9C9D9D9D9E9E9E9F9F9F9F6A
:108C40009F9F9F9E9E9E9D9D9D9C9B9B9A99989762
:108C500096959392908F8D8C8A8886858382818069
:108C6000808183868A9199A2ACB7C1CAD2D9DEE24B
:108C7000E4E5E6E5E4E2E0DEDDE1EBF5F9F8F90054
:108C80000708070B151F2322201E1C1B1A1B1C1E66
:108C900022272E363F49545E676F767A7E7F7F7F2C
:108CA0007F7E7D7B7A7876747371706E6D6B6A6986
:108CB000686766656564646363626262616161617D
:108CC0006161616262626363636465656667686966
:108CD0006A6B6D6E7071737476787A7B7D7E7F7F40
:108CE0007F7F7E7A766F675E54493F362E27221E3D
:108CF0001C1B1A1B1C1E2022231F150B0708070014
:108D00001F313D444E5354565A5F64696E747679F0
:108D10007C7F7F7F7F7F7F7F7F7F7F7F7F7F7F7F66
:108D20007F7F7F7F7F7F7F7F7F7F7F7F7F7F7F7F53
:108D30007F7F7F7F7F7F7F7F7F7F7F7F7F7F7F7F43
:108D40007F7F7F7F7F7F7F7F7F7F7F7F7F7F7F7F33
:108D50007F7F7F7F7F7F7F7F7F7F7F7F7F7F7F7F23
:108D60007F7F7F7F7F7F7F7F7F7F7F7F7F7F7F7F13
:108D70007F7F7F7F7F7F7F7F7F7F7F7C7871684C65
:108D80002C1C120C0A0B0A05FDF3E9DFD4CAC0B78C
:108D9000AEA69E97918B8685828080808080808021
:108DA00080808080808080808080808080808080C3
:108DB00080808080808080808080808080808080B3
:108DC00080808080808080808080808080808080A3
:108DD0008080808080808080808080808080808093
:108DE0008080808080808080808080808080808083
:108DF000808080808087919DACC4CBD4DDF2FAFA6C
:108E000022002400260028002B002D003000330013
:108E1000360039003D004000440048004C0051003D
:108E200056005B00600066006C00730079008100F2
:108E3000880090009900A200AC00B600C100CC00F0
:108E4000D800E500F30001011001210132014401C5
:108E500057016C0181019801B001CA01E5010202CC
:108E60002102410264028802AE02D70203033003EA
:108E700061039403CB03050442048304C704100573
:108E80005D05AF0505066106C206290796070908B4
:108E9000830805098E09200ABA0A5D0B0A0CC10C69
:108EA000840D510E2B0F121007110A121D134014BE
:108EB0007415BA1614188319071BA31C571E2420F7
:108EC0000E22142439267F28E82A752D29300633EE
:108ED0000F364539AD3C49401B442848734CFE5081
:108EE000CF55EA5A51600C661D6C8B725A7992808C
:108EF00037885090E598FDA19FABD3B5A3C0000083
:108F0000382F603CD0F470E0660F771FCB018E5A8B
:108F1000974FFC0124916D5A774FFB016491832F89
:108F200090E0FC0174E0EE0FFF1F7A95E1F7E81B7B
:108F3000F90BE05AF94F21876287832F90E0FC01FB
:108F400054E0EE0FFF1F5A95E1F7E81BF90BE05ACA
:108F5000F94F818523813481280F311D368725877C
:108F6000469546954695842F90E045E0880F991FD9
:108F70004A95E1F7280F391F3487238708951F93F7
:108F8000CF93DF93FA01549131961491C52FD0E01D
:108F90009F012F5F3F4F70E0F5E0660F771FFA9556
:108FA000E1F7680F711D40E00BC084918D939F5FC6
:108FB00031969517D0F34F5F2C0F3D1F605E7F4FAA
:108FC000411730F4DB01A054BE4FF90190E0F1CF1E
:108FD000DF91CF911F9108950F931F93CF93DF934C
:108FE000182FFB01B49131960491CB2FD0E0BF0133
:108FF0006F5F7F4FA0E016C0FA01249190E0FC0162
:10900000EE0FFF1FE80FF91FE050FA4F22833F5F7A
:109010004F5F5F4F832F810F3B1770F31B0FAF5FC5
:109020006C0F7D1FA01718F4AB0130E0F3CFDF9178
:10903000CF911F910F9108950F93A82F70E013C047
:1090400090E0FC01EE0FFF1FE80FF91FE050FA4F10
:10905000508341833F5F585F832F8A0F321780F31D
:10906000A20F7F5F485F701718F4562F30E0F4CFDF
:109070000F9108958093680D10926B0D81E080939D
:109080006A0D662321F080916A0D8823E1F7089527
:10909000982F882319F48FEF87B9089581E0809382
:1090A0006C0D8093690D9093680D10926B0D8093F9
:1090B0006A0D662321F080916A0D8823E1F70895F7
:1090C000982F882311F417B808958CE080936C0DC5
:1090D0008FEF8093690D9093680D10926B0D81E076
:1090E00080936A0D662321F080916A0D8823E1F751
:1090F000089580916A0D8823F9F080916B0D882383
:10910000C1F48091680D80936B0D90916C0DE92FE7
:10911000F0E0E556FE4F808187B98091690D890F97
:1091200080936C0D882311F08D3031F410926A0D0C
:109130000895815080936B0D08950F931F93CF93E3
:10914000DF938C01C0E0D0E007C00E942A39882359
:10915000E1F30E942D392196C017D107B4F3DF91B6
:10916000CF911F910F9108958F929F92AF92BF92CE
:10917000CF92DF92EF92FF920F931F93CF93DF93E3
:10918000882E962E5A016901F02E00E010E080EE44
:10919000F80E0CC0882D8C0F6E2D4F2D0E9451386B
:1091A0002196CA15DB05B4F30F5F1F4F0C151D0583
:1091B0002CF4C0E0D0E0E02EE90CF3CFDF91CF91AA
:1091C0001F910F91FF90EF90DF90CF90BF90AF90E5
:1091D0009F908F90089540520E9451380895FF92B9
:1091E0000F931F93CF93DF938C01F62EEA01FE01BC
:1091F00044912196442349F0802F0F5F1F4F4F77F2
:1092000040526F2D0E945138F2CFDF91CF911F91C4
:109210000F91FF900895FF920F931F93182F062F21
:10922000F42E42954F704A3010F4405F01C0495E01
:10923000812F602F0E9451384F2D4F70812F8F5FEB
:109240004A3010F4405F01C0495E602F0E945138DF
:109250001F910F91FF900895FF920F931F93182F66
:10926000062FF42E452F0E940B49812F8E5F602F11
:109270004F2D0E940B491F910F91FF900895EF927F
:10928000FF920F931F93F62E042F182F88E0E82EDD
:10929000E10E07FF04C0812F6F2D41E103C0812F34
:1092A0006F2D40E10E9451381F5F1E1511F0000F15
:1092B000F0CF1F910F91FF90EF900895DF92EF9202
:1092C000FF920F931F93CF93DF93E62E8A01D22E46
:1092D000EC01FF240115110511F4FF2051F4C80120
:1092E0006AE070E00E949E63482F405F8C2F6E2DD5
:1092F00009C0DD2021F08C2F6E2D40E103C08C2FA2
:109300006E2D40E00E945138F394219785E0F816C5
:1093100039F0C8016AE070E00E949E638B01DACFE9
:10932000DF91CF911F910F91FF90EF90DF90089503
:10933000EF92FF920F931F93CF93DF93F62E042F9C
:10934000E22EEC0110E0002311F4112349F4802FE8
:109350006AE00E949263905F8C2F6F2D492F09C0A5
:10936000EE2021F08C2F6F2D40E103C08C2F6F2D4C
:1093700040E00E9451381F5F2197133031F0802F59
:109380006AE00E949263082FDECFDF91CF911F9198
:109390000F91FF90EF900895CF92DF92EF92FF929E
:1093A0000F931F93CF93DF93C62E79018A01EC01AF
:1093B000DD24E114F1040105110511F4DD2069F447
:1093C000C801B7012AE030E040E050E00E94C563E8
:1093D000462F405F8C2F6C2D03C08C2F6C2D40E0EE
:1093E0000E945138D394219786E0D81669F0C801BD
:1093F000B7012AE030E040E050E00E94C563C901B7
:10940000DA017C018D01D5CFDF91CF911F910F91B2
:10941000FF90EF90DF90CF9008957F928F929F9270
:10942000AF92BF92CF92DF92EF92FF920F931F9372
:10943000CF93DF93782E862E5A016901780100E0E0
:1094400010E00CC0872D8C0F692DA7010E944338B6
:109450002196CA15DB05B4F30F5F1F4F0C151D05D0
:109460002CF4C0E0D0E0902E980CF3CFDF91CF9198
:109470001F910F91FF90EF90DF90CF90BF90AF9032
:109480009F908F907F9008957F928F929F92AF923E
:10949000BF92CF92DF92EF92FF920F931F93CF93E1
:1094A000DF93782E862EEA01FA01C590D490FA0156
:1094B0003296A590B49000E016C0FC01EE0DFF1DA1
:1094C0003296EE0FFF1FEC0FFD1F45915491812F37
:1094D000870D692D0E9443381F5F812F90E08C1506
:1094E0009D055CF30F5F802F90E08A159B055CF46F
:1094F0008C9D70018D9DF00C9C9DF00C112410E052
:10950000902E980CEACFDF91CF911F910F91FF9091
:10951000EF90DF90CF90BF90AF909F908F907F9013
:109520000895FC01DB018FE090E0938382839583B3
:10953000848316968C91169712962C911297829F7F
:10954000C001112411962C911197820F911D9783C0
:1095500086831E968C911E971A962C911A97829F3D
:10956000C001112419962C91820F911D918780873B
:1095700083E0818345878DE2868781E0808B8487C5
:10958000089590E02AE130E0281B390B53E0220FC8
:10959000331F5A95E1F7209371069C0145E0220F95
:1095A000331F4A95E1F740EC51E0240F351F30930B
:1095B00073062093720623E0880F991F2A95E1F71E
:1095C0008093620650936406409363060895FC01FD
:1095D00081818B3E10F48F5F8183908193FF05C062
:1095E00081818B3410F0977F9083908192FF05C02A
:1095F00081818B3410F09B7F90830895FC018185DD
:10960000882321F085818B3408F01186938191FFA6
:1096100005C08681823410F09D7F938386818234D9
:1096200010F48F5F868385818B3410F48F5F858380
:1096300080858F3010F48F5F80870895FC01DB01F7
:1096400080818160808388EB8093710680E292E064
:10965000909373068093720688E18093620680EC93
:1096600091E090936406809363068C91882331F592
:109670001C968D919C911D978C73907088309105EC
:1096800061F08930910518F40497D1F406C0803157
:10969000910561F08097A1F409C08281882319F0B7
:1096A00022E030E00FC021E030E00CC090E0828189
:1096B000882309F491E0928381EF01C08F5F8C933E
:1096C00020E030E0C9010895EF92FF920F931F93BD
:1096D000CF93DF93EC010E94073880E6E0E0F6E0EC
:1096E000DF011D928A95E9F781E30E9460381092AC
:1096F00077068BE59BE19093660680936506109252
:10970000700610926F0680ED8093710680EC91E0F8
:10971000909373068093720610926206909364068B
:10972000809363061A8280E066E045E75EE00E946F
:10973000BF470BE110E0802F8B516AE0A8010E9427
:1097400043380F5F1F4F01331105A9F762E0E62E82
:10975000FF2481E090E00E949D4880E090E06DE071
:1097600070E046E150E02DE030E000E010E00E94C3
:109770000D4A85E090E06EE070E042ED59E00E9415
:10978000EF4885E090E06FE070E04DED59E00E9419
:10979000EF4885E090E060E170E049EE59E00E941A
:1097A000EF486A8170E0625F7F4F83E090E043EFB3
:1097B00059E00E94EF48F3948D819E8101969E832B
:1097C0008D83BFE0FB1629F680E090E02CC080E09E
:1097D0000E9442399C012C7330702830310571F0A1
:1097E0002930310520F424303105E9F407C0203157
:1097F000310559F020323105B1F40EC02A812223FF
:10980000C1F0213081F482E015C02A81222311F0B9
:10981000215006C0EA8207C02A81223018F42F5F47
:109820002A8301C01A828C739070892B09F090CF23
:10983000CECF81E0DF91CF911F910F91FF90EF90FC
:1098400008958F929F92AF92BF92CF92DF92EF9244
:10985000FF920F931F93CF93DF937B01F8E0CF2EFE
:10986000D12CC60ED71E4B01EC018C01015B1F4FA2
:10987000AA24BB248C8585FF2AC0698170E06D5FB6
:109880007F4F4A8150E0425F5F4FC7010E942E5ACE
:109890008823E9F4F801218130E0F701848590E024
:1098A000E3E0880F991FEA95E1F7FE0132968217EF
:1098B00093075CF481E0B601AF010E940D59882343
:1098C000F1F1F8018181815033C081E034C08C8591
:1098D00084FF35C0698170E06D5F7F4F4A8150E041
:1098E000455F5F4FC7010E942E5A882341F5F8015A
:1098F000418150E0F701238530E0265030408485D7
:1099000090E0BC01269FC001279F900D369F900DCF
:109910001124FE0132964817590764F480E0B6011D
:10992000AF010E940D59882351F0F80181818F5FAA
:10993000818305C080E0BF01A6010E94A0598C85EB
:1099400086FF31C0698170E06F5F7F4F4A8150E0D0
:10995000435F5F4FC7010E942E5A882321F5F8010B
:10996000408150E0F701238130E02650304084816F
:1099700090E0BC01269FC001279F900D369F900D5F
:109980001124FE013196481759075CF480E0B401B8
:10999000AF010E940D598823B9F1F80180818F5FD2
:1099A0002CC080E02DC08C8587FF2EC0698170E0BF
:1099B0006B5F7F4F4A8150E0435F5F4FC7010E945A
:1099C0002E5A882309F5F801208130E0F7018481BF
:1099D00090E073E0880F991F7A95E1F7FE013196C8
:1099E0008217930764F481E0B401AF010E940D591E
:1099F000882351F0F80180818150808305C081E087
:109A0000BF01A4010E94A0598C859D8593FF03C0CE
:109A1000CE010E94E6628C859D8592FF07C08885F5
:109A20008F3020F0CE010E94D35F18860894A11CCD
:109A3000B11CC25BDF4F0E541040F2E0AF16B10410
:109A400009F018CFDF91CF911F910F91FF90EF9008
:109A5000DF90CF90BF90AF909F908F9008950F931D
:109A60001F93CF93DF93EC018B018C8585FF15C08D
:109A7000698170E06D5F7F4F4A8150E0425F5F4FC8
:109A8000C8010E942E5A882341F4B801685F7F4FB5
:109A9000AE014E5F5F4F81E016C08C8584FF15C01C
:109AA000698170E06D5F7F4F4A8150E0455F5F4F95
:109AB000C8010E942E5A882341F4B801685F7F4F85
:109AC000AE014E5F5F4F0E940D598C8586FF11C01D
:109AD000698170E06F5F7F4F4A8150E0435F5F4F65
:109AE000C8010E942E5A882321F4AE014F5F5F4FB8
:109AF00014C08C8587FF14C0698170E06B5F7F4F55
:109B00004A8150E0435F5F4FC8010E942E5A88236C
:109B100039F4AE014F5F5F4F81E0B8010E940D59EB
:109B20008C859D8593FF03C0CE010E94E6628C85E3
:109B30009D8592FF07C088858F3020F0CE010E945E
:109B4000D35F1886DF91CF911F910F910895FC018B
:109B5000178691E0908B848585FF03C0168684E18B
:109B600004C084FF03C0968781E18787848586FFD0
:109B700004C082E0868785E005C087FF04C083E0DB
:109B800086878BE087878485958583709370823084
:109B9000910521F18330910518F40197D9F508C09A
:109BA00021E08030920741F18050924099F50FC03A
:109BB0008685823031F0833031F0813031F484E1B8
:109BC00003C088E001C08EE08787168623C08685A3
:109BD000882311F481E1878781E01BC08685882373
:109BE00011F481E187878685833021F48FEF808BA4
:109BF00085E0878782E00DC08685882311F481E1A6
:109C000087878685823021F48FEF808B8BE0878772
:109C100083E08687CF010E960E94FF5108950F932F
:109C20001F938C0184E70E94603888ED9EE30E94B8
:109C3000E13B86E1F801838386E0848380E38683C9
:109C400080E1858398E097838AE18387948780E227
:109C50008687858784E087871282128681E08093D9
:109C600077068BEC9EE090937506809374061092B5
:109C7000700610926F0610926806909366068093A5
:109C800065061092020681E00E9468388FE7F801AD
:109C90008083808780E0608940E220E20E94B253A6
:109CA000C8010E94CB561F910F9108952F923F92A9
:109CB0004F925F926F927F928F929F92AF92BF92DC
:109CC000CF92DF92EF92FF920F931F93CF93DF9388
:109CD0005C01E62ED72EF42E49010E940738D401EC
:109CE00015968D919C9116970E94656381E1F5010F
:109CF00011928A95E9F72EE4FF2DF20290011124CA
:109D00008E2D9D2D60E070E0A9010E9482638DE49C
:109D1000D4011D928A95E9F78AEAF80111928A9591
:109D2000E9F780E6E0E0F6E0DF011D928A95E9F7C9
:109D3000F501F08AC5010E940F4ED50150962C9175
:109D400030E08AE190E0821B930B53E0880F991F6B
:109D50005A95E1F780937106C90145E0880F991F74
:109D60004A95E1F780549E4F909373068093720654
:109D700083E0220F331F8A95E1F72093620680EC7F
:109D800091E090936406809363068E2D9D2DEC01E7
:109D9000BE01685B7F4FEE24FF24B8E4CB2EDD24A8
:109DA000D39451E0A0E44A2EF6EA6F2E712CE3E240
:109DB0005E2E49E1242E34E0332E8EC0D98A1C8ACF
:109DC0005A8B8D2D90E0FC01EE0FFF1FE80FF91F5D
:109DD000E050FA4F5283898990E00196FC01EE0F22
:109DE000FF1FE80FF91FE050FA4F565F52835A5099
:109DF000298930E04981C9010196FC01EE0FFF1F5E
:109E0000E80FF91FE050FA4F4083F901EE0FFF1FF2
:109E1000E20FF31FE050FA4F4083898990E0FC0184
:109E2000EE0FFF1FE80FF91FE050FA4F8A81818380
:109E3000898990E00196FC01EE0FFF1FE80FF91FE2
:109E4000E050FA4F8A81885F8183DE01569620E0D8
:109E500089898E5F820F1C968C931C971D964C925D
:109E60001D9714967C926E92139712967C926E9226
:109E70001197E5E0EC9390E0FC01EE0FFF1FE80F77
:109E8000F91FE050FA4F42822F5F5196233001F7BD
:109E9000C982F6EAFA8328835F82E4E6DB01119641
:109EA000EC93119712965C921297FFE3FC93149631
:109EB0002C92149715963C92159780E413968C93E8
:109EC0000894E11CF11CC25BDF4F9AE0C90E625B93
:109ED0007F4FA5E0DA0E5A5EF501808990E0E81622
:109EE000F9060CF46BCF81E090E0D40114969C93BA
:109EF0008E9313978FE090E0F8019383828395838C
:109F00008483D50116968C91169712962C911297F0
:109F1000829FC001112411962C911197820F911DDF
:109F2000978386831E968C911E971A962C911A976A
:109F3000829FC001112419962C91820F911D918747
:109F4000808783E081838BE085878DE2868781E04F
:109F5000808B8487DF91CF911F910F91FF90EF90BD
:109F6000DF90CF90BF90AF909F908F907F906F9039
:109F70005F904F903F902F9008952F923F925F9265
:109F80006F927F928F929F92AF92BF92CF92DF9209
:109F9000EF92FF920F931F93DF93CF93CDB7DEB76E
:109FA000C755D1400FB6F894DEBF0FBECDBF4C01F0
:109FB000A2E1EA2EF12CEC0EFD1EFEEAAF2EB12C32
:109FC000AC0EBD1E6E010894C11CD11CC601B701A8
:109FD00042E0940185010E94564E5E2C6F2CE0E613
:109FE0002E2E312C2C0E3D1E7C2CCD2C76EAD72E1D
:109FF00081E090E00E949D48C401652D762D0E946D
:10A000002154C4010E94E74A852D962D0E94FE4AE4
:10A0100080E00E9442399F8F8E8FC1010E94FE4ACC
:10A0200081E00E944239282FAD968FAFAD97AE9652
:10A030009FAFAE978A8918168CF0F10180811816AF
:10A040006CF0C401652D762D0E941E4B8130910568
:10A0500009F492C00297A1F480E08FC08E8D82FD3A
:10A0600002C022FF0DC0F40181818F3048F01182BF
:10A07000808180FF02C08E7F02C08160F4018083F6
:10A08000F401808180FD71C08A8918165CF4F101A9
:10A09000808118164CF4852D962D672D7C2D0E94FD
:10A0A000214C08C0C10102C0852D962D672D7C2D45
:10A0B0000E942F4D8A8180936F068A858093700657
:10A0C0008981882319F48985882321F0872D9C2D87
:10A0D0000E94CB56872D9C2DB4010E949B58C50130
:10A0E000672D7C2DA401252D362D0E94095F872D1B
:10A0F0009C2DB401452D562D0E94D75A852D962DA5
:10A100008C0163E0E62E66E0F62EC8010E94A74DA2
:10A11000F80187818F5F8783872D9C2DB401A8016B
:10A1200095010E944762F801838181FF04C0F40118
:10A13000858181FF0CC0F8018181F70183838083D1
:10A14000F8018281F7018183885F848305C0F7016C
:10A15000D382D082D182D482025B1F4F8FE090E005
:10A16000E80EF91E0A151B0581F6F401858196811A
:10A170000196968385833CCF82E0C95ADE4F0FB6A5
:10A18000F894DEBF0FBECDBFCF91DF911F910F912D
:10A19000FF90EF90DF90CF90BF90AF909F908F9007
:10A1A0007F906F905F903F902F9008958F929F9235
:10A1B000AF92BF92CF92DF92EF92FF920F931F93D5
:10A1C000DF93CF93CDB7DEB7C950D1400FB6F89427
:10A1D000DEBF0FBECDBF4C0102E1E02EF12CEC0E34
:10A1E000FD1E10E6A12EB12CAC0EBD1E6E01089412
:10A1F000C11CD11CC601B70141E0940185010E9438
:10A20000564E1E2DEF2C0C2DCD2CDA2CAB2CB6EA95
:10A21000FB2E81E090E00E949D48C401612F7E2DBD
:10A220000E943355C4010E94E74A812F9E2D0E944F
:10A23000FE4A80E00E944239282F8E8F9F8F8A89A4
:10A2400018166CF0C401612F7E2D0E941E4B8130C8
:10A25000910509F474C0029789F480E071C022FF6F
:10A260000DC0F40181818F3048F01182808180FF20
:10A2700002C08E7F02C08160F4018083F40180817E
:10A2800080FD56C0812F9E2D602F7C2D0E942F4D6A
:10A290008A8180936F068A858093700689818823DE
:10A2A00019F48985882321F0802F9C2D0E94CB569C
:10A2B000802F9C2DB4010E949B58812F9E2D0E94BF
:10A2C000A74D898D8F5F898F802F9C2DB401412FE1
:10A2D0005E2D2D2D3A2D0E944762802F9C2DB401BA
:10A2E000412F5E2D0E94D75A8D2D9A2D602F7C2DE7
:10A2F000A401212F3E2D0E94095F8D8981FF04C09A
:10A30000F401858181FF0CC08B89809306068093C0
:10A3100003068C8980930406885F8093070608C033
:10A32000F0920606F0920306F0920406F0920706F9
:10A33000F401858196810196968385836ACF81E0B9
:10A34000C75FDE4F0FB6F894DEBF0FBECDBFCF9113
:10A35000DF911F910F91FF90EF90DF90CF90BF9012
:10A36000AF909F908F9008950F931F93DF93CF939B
:10A37000CDB7DEB7CD54D0400FB6F894DEBF0FBED8
:10A38000CDBF8BE290E30E946338FE0131968DE4ED
:10A39000DF011D928A95E9F780E08F01813049F055
:10A3A000813018F08230D1F708C0C8010E94644B98
:10A3B000F5CFC8010E94D650F1CFC8010E94BD4F11
:10A3C000EDCFCF93DF93EC0150E020E030E011C0FF
:10A3D000FE01E20FF31F85919591A591B491FB01C8
:10A3E000E20FF31F80839183A283B3835F5F2C5FAF
:10A3F0003F4F541768F3CB01DF91CF910895DC01F3
:10A4000011968C9111978823C1F416968C9116970A
:10A41000882319F016961C92169713968C91139711
:10A4200090E0FC01EE0FFF1FE80FF91FE050FA4F1C
:10A430008C9114969C91890F66C015968C911597F6
:10A440008430A0F015961C92159716969C9116973D
:10A45000892F8E5F853010F080E004C012968C91B9
:10A460001297890F16968C93169704C08F5F1596D6
:10A470008C93159713968C91139790E0FC01EE0F37
:10A48000FF1FE80FF91FE050FA4F8C9114969C9132
:10A490001497890F828313968C91139790E00196FD
:10A4A000FC01EE0FFF1FE80FF91FE050FA4F119665
:10A4B0008C91119714969C911497890F828313960F
:10A4C0008C911397282F30E02F5F3F4FF901EE0F4B
:10A4D000FF1FE20FF31FE050FA4F428116969C9146
:10A4E0001697933039F09D3F29F012968C91981B66
:10A4F000892F01C080E0F901EE0FFF1FE20FF31F6B
:10A50000E050FA4F840F82830895DC0112968D91FA
:10A510009C9113978F3F910509F060F414962D914B
:10A520003C9115972F3F310509F024F497FD02C0A7
:10A53000482F02C046EA26EA11968C911197853081
:10A54000F1F087FD1CC01D968C911D9790E001963F
:10A55000FC01EE0FFF1FE80FF91FE050FA4F285FD4
:10A56000218328501D968C911D9790E00196FC0147
:10A57000EE0FFF1FE80FF91FE050FA4F40831D96C2
:10A580008C911D9790E0FC01EE0FFF1FE80FF91F63
:10A59000E050FA4F40831D968C9190E0FC01EE0F45
:10A5A000FF1FE80FF91FE050FA4F218308957F92B3
:10A5B0008F929F92AF92BF92CF92DF92EF92FF92D3
:10A5C0000F931F93CF93DF93B82ED62E7A014A01B3
:10A5D000892C992482940FE08022CA019695879550
:10A5E00096958795B7E07B2E7822072D0B0DCA0133
:10A5F000A5E096958795AA95E1F7182F1770C12EBB
:10A60000C60EC0E0D0E06C2FAE01427050707C2FBF
:10A610007170CA010296880F991F272F2F5F282B70
:10A6200030E0282139212330310520F42130310553
:10A6300040F40EC02430310559F02830310591F432
:10A6400007C066956C0D55954795465F5F4F07C0EF
:10A6500066956C0DAE0141705070485F5F4F872F5B
:10A66000800F06C066956C0D872F800F4CE050E080
:10A670000E9443382196C430D10529F6F7FE1DC04B
:10A6800082E0D80E1D0D8EEFD80EA02EA394CD2DF6
:10A69000D0E023960DC0802F612F48E050E00E944B
:10A6A00043388A2D612F49E050E00E9443381F5FF4
:10A6B000812F90E0C817D90774F7F6FE12C0A02EBC
:10A6C000A3941C2D1150802F612F48E050E00E9470
:10A6D00043388A2D612F49E050E00E944338D1165B
:10A6E00088F3F5FE1EC082E0B80E1B2D170D8EEF0D
:10A6F000B80EDC2CD394CB2DD0E027960DC0812F43
:10A700006C2D4AE050E00E944338812F6D2D4BE0C4
:10A7100050E00E9443381F5F812F90E0C817D9078F
:10A7200074F7F4FE11C01C2D1F5F0150802F6C2D9B
:10A730004AE050E00E944338802F612F4BE050E008
:10A740000E944338B01688F3DF91CF911F910F918B
:10A75000FF90EF90DF90CF90BF90AF909F908F9041
:10A760007F900895BF92CF92DF92EF92FF920F9366
:10A770001F93CF93DF93B62E082FE82EFF24E40E0D
:10A78000F11CC62FD0E0C20FD11D11C04170507016
:10A79000440F551F4C295D29802F612F0E9443389B
:10A7A0001F5F412F50E04C175D0784F30F5F802F30
:10A7B00090E08E159F053CF41B2D21E0C22ED12C7C
:10A7C000C822D922EECFDF91CF911F910F91FF9038
:10A7D000EF90DF90CF90BF900895DC01FB01808166
:10A7E000482F50E012968C911297481B510983E034
:10A7F000440F551F8A95E1F78281480F511D9181C1
:10A800001A968C911A97638140325105CCF4292F06
:10A8100030E0281B3109220F331F220F331F260F70
:10A82000311D2032310564F457FD0AC037FD08C0E0
:10A8300050966C91620F842F41E021E00E94B25348
:10A840000895CF92DF92EF92FF920F931F93CF93D1
:10A85000DF936C017B0180E090E060E070E048E114
:10A8600050E022E030E00DE010E00E940D4A80E070
:10A8700060E041E450E00E944338F701428553858F
:10A8800085E090E060E070E021E00E945E49F70121
:10A89000848190E0FC01EE0FFF1FE80FF91FEE0D21
:10A8A000FF1DE75BFF4F8AE090E060E070E04081D1
:10A8B00021E00E949849F701848190E0FC01EE0FAD
:10A8C000FF1FE80FF91FEE0DFF1DE85BFF4F4081F2
:10A8D00088E060E050E00E9443388BE060E041E4B3
:10A8E00050E00E944338E701C25BDF4F4A855B8539
:10A8F00080E190E060E070E021E00E945E498C81A0
:10A9000090E0FC01EE0FFF1FE80FF91FEC0FFD1F99
:10A91000E75BFF4F85E190E060E070E0408121E07F
:10A920000E9498498C8190E0FC01EE0FFF1FE80F18
:10A93000F91FEC0FFD1FE85BFF4F408183E160E0F2
:10A9400050E00E944338F701808118168CF188810D
:10A95000181674F180E090E061E070E048E150E0AA
:10A9600022E030E00E940D4A88E090E062E070E072
:10A9700040EE5FE30E94EF4881E090E061E070E02C
:10A980004AEE5FE30E94EF4881E090E062E070E011
:10A9900041EF5FE30E94EF48F601628170E06F5F74
:10A9A0007F4F80E090E047EF5FE30E94EF4852C0A6
:10A9B000E701FF24F601808190E080FF0BC084E076
:10A9C00090E061E070E042EC5FE30E94EF4800E05D
:10A9D00010E031C09C012C70307021153105B9F3A5
:10A9E000F601858181FFF3CF2830310569F02C30E5
:10A9F000310589F02430310551F783E090E061E0C2
:10AA000070E049EC5FE3E1CF83E090E061E070E06B
:10AA100041ED5FE3DACF83E090E061E070E048ED84
:10AA20005FE3D3CF8F2D800F61E04EE050E00E94B6
:10AA300043380F5F1F4F8881992787FD909508172E
:10AA4000190784F3C25BDF4FFBE0FF0E86E1F816C7
:10AA500009F0B0CFDF91CF911F910F91FF90EF9050
:10AA6000DF90CF900895EF92FF920F931F93CF93B3
:10AA7000DF937C01EB0180E090E060E070E048E172
:10AA800050E021E030E00DE010E00E940D4A80E14E
:10AA900060E041E450E00E9443384A855B8585E1EF
:10AAA00090E060E070E021E00E945E498C8190E0DF
:10AAB000FC01EE0FFF1FE80FF91FEC0FFD1FE75B16
:10AAC000FF4F8EE090E060E070E0408121E00E9466
:10AAD00098498C8190E0FC01EE0FFF1FE80FF91FF1
:10AAE000EC0FFD1FE85BFF4F40818CE060E050E021
:10AAF0000E9443388881181674F180E090E061E08C
:10AB000070E048E150E022E030E00E940D4A80E031
:10AB100090E060E070E040EE5FE30E94EF4885E087
:10AB200090E061E070E04AEE5FE30E94EF4885E06C
:10AB300090E062E070E041EF5FE30E94EF48F701D0
:10AB4000628170E06F5F7F4F84E090E047EF5FE3EA
:10AB50000E94EF4847C0F701808190E080FF0BC062
:10AB600084E090E060E070E042EC5FE30E94EF4838
:10AB700000E010E030C09C012C70307021153105D0
:10AB8000B9F3F701858181FFF3CF2830310569F0F2
:10AB90002C30310589F02430310551F783E090E005
:10ABA00060E070E049EC5FE3E1CF83E090E060E0DB
:10ABB00070E041ED5FE3DACF83E090E060E070E0C9
:10ABC00048ED5FE3D3CF802F60E04EE050E00E947D
:10ABD00043380F5F1F4F8881992787FD909508178D
:10ABE00019078CF3DF91CF911F910F91FF90EF9098
:10ABF00008959F92AF92BF92CF92DF92EF92FF9211
:10AC00000F931F93CF93DF93082F162F5A01DD2444
:10AC100063E0962E910E52E0C52EC80ECD2DD0E0E9
:10AC2000CC0FDD1FCA0DDB1D68817981872F992725
:10AC30008F709070019791F47695679576956795EA
:10AC4000862F877093E0769567959A95E1F7677000
:10AC5000610F800F46E25EE00E94BF474881598144
:10AC6000E52EFF24C7018F709070029721F4802F8A
:10AC7000612F0E94D75268817981872F99278F7021
:10AC80009070039791F47695679576956795862FE2
:10AC90008770F3E076956795FA95E1F76770610F35
:10ACA000800F4CE25EE00E94BF4768817981872F68
:10ACB00099278F709070049731F576956795769502
:10ACC0006795862F877043E0769567954A95E1F7FB
:10ACD0006770690D800F4FE35EE00E94BF47688197
:10ACE00079817695679576956795862F877023E0AD
:10ACF000769567952A95E1F76770610F8C0D47E3AC
:10AD00005EE00E94BF4768817981872F99278F7005
:10AD10009070059791F47695679576956795862F4F
:10AD20008770B3E076956795BA95E1F76770610F24
:10AD3000800F47E45EE00E94BF4768817981872FDA
:10AD400099278F709070069791F476956795769510
:10AD50006795862F8770E3E076956795EA95E1F72A
:10AD60006770610F800F41E65EE00E94BF478881F7
:10AD7000998183709070892B11F4D3944FCFDF9118
:10AD8000CF911F910F91FF90EF90DF90CF90BF90E8
:10AD9000AF909F9008956F927F928F929F92AF9203
:10ADA000BF92CF92DF92EF92FF920F931F93DF93A8
:10ADB000CF93CDB7DEB76D970FB6F894DEBF0FBE59
:10ADC000CDBF8C01DC0118968C91882311F490E0A2
:10ADD00083C08F3F91F4F801808990E055E0880F9F
:10ADE000991F5A95E1F7BC0160547E4F805C9D4FDE
:10ADF00040E853E00E94706302C0813011F090E09F
:10AE000013C0D80150968C9190E035E0880F991FBF
:10AE10003A95E1F7BC01605C7D4F80549E4F40E85D
:10AE200053E00E94706397E0992E990C990CF801F9
:10AE30006089690D80E040E224E09D8F0E94B2535A
:10AE4000EE24FF249D8DC92EDD245E010894A11CF3
:10AE5000B11C7E2DD80112968C911297F701E80F44
:10AE6000F11D85E0EE0FFF1F8A95E1F71A968C9190
:10AE70001A979601280F311DE20FF31FEE0FFF1FE7
:10AE8000EA5DF54F4591549150966C9120E030E089
:10AE9000F901E40FF51F85919591A591B491F50104
:10AEA000E20FF31F80839183A283B3832C5F3F4F14
:10AEB0002C30310569F7690D872F880F880F880FAF
:10AEC000A5010E94F9550894E11CF11C34E0E31639
:10AED000F10409F0BECF94E0D8018C91882309F4E5
:10AEE00092C08F3F99F450968C9190E055E0880F76
:10AEF000991F5A95E1F7BC0160547E4F88539E4FCD
:10AF000048EF53E00E94706390E014C0813091F4E8
:10AF1000F801808990E035E0880F991F3A95E1F7B4
:10AF2000BC0168537E4F80549E4F48EF53E00E940F
:10AF3000706393E0C92ECC0CCC0CCC0C8C2DD801BA
:10AF400050966C9148E020E29D8F0E94B253F80128
:10AF50008281282F30E09D8D290F311D95E0220F31
:10AF6000331F9A95E1F78285280F311D220F331F79
:10AF70002A5D354F40E050E0BE01635F7F4FF9012D
:10AF8000E40FF51F85919591A591B491FB01E40F14
:10AF9000F51F80839183A283B3834C5F5F4F403161
:10AFA000510569F77B01DD245E010894A11CB11CE9
:10AFB000D80150967C91F7014081518120E030E02A
:10AFC000FA01E20FF31F85919591A591B491F501D6
:10AFD000E20FF31F80839183A283B3832C5F3F4FE3
:10AFE0002C30310569F76D2D660F660F670F8C2DBC
:10AFF000A5010E94F955D39422E030E0E20EF31E41
:10B0000038E0D316A9F6D80118968C9118978F3787
:10B0100009F077C08C918F3709F073C050962C914E
:10B0200080E0622F40E2205E0E94B253CC24DD24F7
:10B03000BDE06B2E712C6C0E7D1E4E010894811CA0
:10B04000911C6C2DF80182819601280F311DA5E01D
:10B05000220F331FAA95E1F78285280F311D220F99
:10B06000331F2A5D354F40E050E0F901E40FF51F32
:10B0700085919591A591B491F301E40FF51F80831B
:10B080009183A283B3834C5F5F4F4031510569F7D1
:10B09000A62EAA0CAA0CAA0C7301BB24D8015096A8
:10B0A0007C91F7014081518120E030E0FA01E20F0C
:10B0B000F31F85919591A591B491F401E20FF31FCF
:10B0C00080839183A283B3832C5F3F4F2C30310563
:10B0D00069F76B2D660F660F670F8A2DA4010E941A
:10B0E000F955B39422E030E0E20EF31E38E0B316D7
:10B0F000A9F60894C11CD11C84E0C816D10409F03B
:10B10000A0CFD80118961C9218971C926D960FB676
:10B11000F894DEBF0FBECDBFCF91DF911F910F918D
:10B12000FF90EF90DF90CF90BF90AF909F908F9067
:10B130007F906F900895CF92DF92EF92FF920F93DE
:10B140001F93CF93DF937C016B01EB0100E010E0D4
:10B150008B85882309F451C08F81A82FB0E0F701B7
:10B160008281A81BB10993E0AA0FBB1F9A95E1F752
:10B170008985A80FB11D988582854A85A032B105C1
:10B18000E4F5292F30E0281B3109220F331F220F4D
:10B19000331F240F311D203231057CF5B7FD2DC042
:10B1A00037FD2BC06089F901E60FF11D75E0EE0F48
:10B1B000FF1F7A95E1F7EA0FFB1FE054FE4FE08195
:10B1C000E430A8F08C85E81791F0C80163E0880F9F
:10B1D000991F6A95E1F7801B910B07968C0D9D1DB9
:10B1E000FC0187E0DF011D928A95E9F70DC0620F2F
:10B1F0004C858A2F50E00E9443380F5F1F4F2796DF
:10B200000A30110509F0A4CFDF91CF911F910F9162
:10B21000FF90EF90DF90CF900895AF92BF92CF92C2
:10B22000DF92EF92FF920F931F93CF93DF93FB0177
:10B230006A01DA014C915481882309F44EC0A42E8E
:10B24000BB248381C82FD0E0E52EFF242697CE9D16
:10B25000C001CF9D900DDE9D900D11242696A8165D
:10B26000B90614F44F5F5FC01181812F90E020E296
:10B2700030E02C1B3D0BB9016E9D90016F9D300D90
:10B280007E9D300D1124821793071CF41F5F1183DC
:10B2900044C00281202F30E0678180EE9FEF70E094
:10B2A0000E94B2638581680F711D261737074CF421
:10B2B0000F5F02831F5F8681181B118381E08083EB
:10B2C00034C0EC9EC001ED9E900DFC9E900D1124AB
:10B2D000A816B9064CF54F5F25C0242F30E0852F06
:10B2E00090E063E0880F991F6A95E1F78217930752
:10B2F00024F44150F601408317C08181882319F05E
:10B30000815081830AC08281882349F081508283E1
:10B310008681815081838FEF808381E006C054173E
:10B3200018F44150D6014C9380E0DF91CF911F91EA
:10B330000F91FF90EF90DF90CF90BF90AF90089566
:10B34000DB01FA01882371F05C91852F90E0248164
:10B350004381249F90011124821793071CF45F5F9F
:10B360005C9308959C918481891710F491509C936B
:10B370000895DC01FB0116968D919C91179712960A
:10B380002D913C911397820F931F2181821B91096C
:10B3900026814281249F90011124821B930B1396D6
:10B3A0009C938E93129718968D919C911997149651
:10B3B0002D913C911597820F931F2185821B910936
:10B3C00026854285249F90011124821B930B15969C
:10B3D0009C938E93149786812281829FC0011124B1
:10B3E0002181820F911D17969C938E9316978685C7
:10B3F0002285829FC00111242185820F911D1996FB
:10B400009C938E9318970895EF92FF920F931F933A
:10B41000FC018B017A012181DB018D919C9164817A
:10B42000820F911D70E00E94B26361507040D8019C
:10B430006D937C932185D7018D919C916485820FBA
:10B44000911D70E00E94B26361507040F7017183FA
:10B4500060831F910F91FF90EF900895DF93CF933A
:10B4600000D000D0CDB7DEB77A8369835C834B838D
:10B47000BE016F5F7F4FAE014D5F5F4F0E94045A68
:10B48000EB81FC8175E0EE0FFF1F7A95E1F7898172
:10B490009A81E80FF91FE054FE4FE0818E2F84500F
:10B4A000843060F08FE0E81721F4E43238F482E071
:10B4B00006C08F5F8F33B9F780E001C081E00F9045
:10B4C0000F900F900F90CF91DF910895EF92FF9220
:10B4D0000F931F93DF93CF9300D000D0CDB7DEB78B
:10B4E0007C01FB018A01818189831A82828190E03B
:10B4F00008969C838B83C701BE016F5F7F4FAE01AF
:10B500004D5F5F4F0E94045AF801808190E0F7017F
:10B510002281821B9109F3E0880F991FFA95E1F7C8
:10B52000F8012281820F911D29813A81281739075C
:10B5300011F040E016C040E0F801818190E0F70191
:10B540002285821B9109880F991F880F991FF80186
:10B550002381820F911D2B813C812817390709F423
:10B5600041E0842F0F900F900F900F90CF91DF91BB
:10B570001F910F91FF90EF9008950E94606360E02B
:10B5800074E00E94B2639C0109C02E5F3F4F329667
:10B5900083E02F3B380728F020E030E0F901E05449
:10B5A000FE4F80818450843080F7C90108952F9226
:10B5B0003F924F925F926F927F928F929F92AF9243
:10B5C000BF92CF92DF92EF92FF920F931F93CF9390
:10B5D000DF933C015B012A010E94606368EE73E027
:10B5E0000E94B263875B9340C4F1F501C0E0D0E0F4
:10B5F00083858823C9F50E9460638E0123E0000FD4
:10B60000111F2A95E1F70C1B1D0B0A0D1B1D60E194
:10B6100070E00E94B263D80117968C930E94606319
:10B6200060E270E00E94B263F80180870E9460636C
:10B6300068E070E00E94B263D80119968C930E9472
:10B64000606364E070E00E94B263F801828781E089
:10B65000838784E1858782E48487992404E6202E09
:10B66000312C17E0812E4CC021963796CA30D10577
:10B6700009F0BECFF2CFD7011B968C918823A9F198
:10B68000E801B3E0CC0FDD1FBA95E1F7C01BD10B89
:10B690002796CA0DDB1DC301B601AE010E94665A92
:10B6A000882319F1F701838590E0FC01EE0FFF1F5D
:10B6B000E80FF91FEC0DFD1DE75BFF4F5081D7012F
:10B6C0001D964C91252F30E0C101841B910928174C
:10B6D00039075CF4450F4083C301BE010E94ED535E
:10B6E000FE01282D11922A95E9F70F5F1F4F87E081
:10B6F00090E0E80EF91E0A30110509F0BCCF9394D2
:10B70000D30150968C91981650F4BEE49B9E600134
:10B710001124C40CD51C750100E010E0ACCFDF9102
:10B72000CF911F910F91FF90EF90DF90CF90BF903E
:10B73000AF909F908F907F906F905F904F903F90D1
:10B740002F900895DC0111969C911197933071F51B
:10B750001D962C911D9730E0C9010196FC01EE0F5A
:10B76000FF1FE80FF91FE050FA4F46EA4083F90146
:10B77000EE0FFF1FE20FF31FE050FA4F40831D96BC
:10B780008C9190E09C012F5F3F4FF901EE0FFF1F5E
:10B79000E20FF31FE050FA4F4183FC01EE0FFF1F51
:10B7A000E80FF91FE050FA4F418308951F968C91DE
:10B7B0001F97863041F41F961C921F979F5F11962A
:10B7C0009C93119704C08F5F1F968C931F971D96B3
:10B7D0008C911D9790E0FC01EE0FFF1FE80FF91F01
:10B7E000E050FA4F1E968C911E97845F11969C91A3
:10B7F0001197890F82831D968C911D9790E0019679
:10B80000FC01EE0FFF1FE80FF91FE050FA4F1E96E4
:10B810008C911E97815F11969C91890F8283089568
:10B820000F931F93CF93DF93EC018B01CB010E9409
:10B83000BD5AAC019C012F7130702F5F3F4FC90181
:10B84000880F991F820F931F880F991FF80121817C
:10B85000821B91099B838A8375E0569547957A955B
:10B86000E1F74F5F5F4F63E0440F551F6A95E1F7C3
:10B870008185481B51095D834C8304C02E5F3F4F77
:10B880003D832C836A817B816B5F7F4F4C815D811F
:10B89000435F5F4FC8010E942E5A2C813D8188234F
:10B8A00069F78EEE89832F5F3F4F3D832C838DE2B6
:10B8B0008E8781E0888B8C87DF91CF911F910F91CC
:10B8C00008950F931F93CF93DF93EC018B01FB013E
:10B8D000A381B481AA30B10520F0FC0120E030E062
:10B8E00033C0CD0124E0880F991F2A95E1F78A0F14
:10B8F0009B1F8C0F9D1FBA010E94105CF801838171
:10B900009481FC01A4E0EE0FFF1FAA95E1F7E80F78
:10B91000F91FEC0FFD1F7197858571968E5F8587E6
:10B92000F8018381948101969483838310C01E2F34
:10B930009F2F81817196833029F4812FBA010E9453
:10B94000105C05C02F5F3F4F2A173B0780F3DF9144
:10B95000CF911F910F910895CF93DF93EC01DB01FD
:10B960008D8590E0FC01EE0FFF1FE80FF91FE050FE
:10B97000FA4F2E852C5E8981992787FD9095039734
:10B9800095958795959587958170280F22833981A4
:10B990003E30C4F08D8590E00196FC01EE0FFF1F54
:10B9A000E80FF91FE050FA4F2E852C5E832F992760
:10B9B00087FD9095039795958795959587958170C7
:10B9C000280F22838981853164F08D8590E0FC0108
:10B9D000EE0FFF1FE80FF91FE050FA4F86EA818350
:10B9E00080838A858130C9F0813030F0823041F126
:10B9F000833009F048C035C06A817B816D5F7F4F1D
:10BA00004C815D81455F5F4FCD010E942E5A882396
:10BA1000D1F58C819D81019710C06A817B816D5F1A
:10BA20007F4F4C815D81425F5F4FCD010E942E5A56
:10BA3000882349F58C819D8101969D838C8323C049
:10BA40006A817B816F5F7F4F4C815D81435F5F4F78
:10BA5000CD010E942E5A8823B1F48A819B810197DF
:10BA600010C06A817B816B5F7F4F4C815D81435F3A
:10BA70005F4FCD010E942E5A882329F48A819B8131
:10BA800001969B838A8389818F5F89838A3111F430
:10BA900083E08983DF91CF910895AF92BF92CF92D7
:10BAA000DF92EF92FF920F931F93CF93DF93EC01FE
:10BAB000CB018A0179016A0157FF04C0CC24DD243F
:10BAC000C41AD50A5701F7FE04C0AA24BB24AE1835
:10BAD000BF08AC14BD040CF045C010161106FCF4F0
:10BAE0006A817B816F5F7F4F4C815D81435F5F4FD8
:10BAF0000E942E5A882331F48A819B8101979B836F
:10BB00008A8309C08C819D81F7FC02C0019701C026
:10BB100001969D838C8382E08A8785E064C001154D
:10BB2000110509F461C06A817B816B5F7F4F4C8195
:10BB30005D81435F5F4F0E942E5A882331F48A81D2
:10BB40009B8101969B838A8309C08C819D81F7FC30
:10BB500002C0019701C001969D838C8383E08A8790
:10BB600088E041C01E141F04ECF46A817B816D5F84
:10BB70007F4F4C815D81455F5F4F0E942E5A882325
:10BB800031F48C819D8101979D838C8309C08A81CA
:10BB90009B8117FD02C0019701C001969B838A8398
:10BBA0001A8620C0E114F104F9F06A817B816D5F8F
:10BBB0007F4F4C815D81425F5F4F0E942E5A8823E8
:10BBC00031F48C819D8101969D838C8309C08A818B
:10BBD0009B8117FD02C0019701C001969B838A8358
:10BBE00081E08A878BE08B87CA18DB080894C11C28
:10BBF000D11C83E0C816D10490F41016110614F479
:10BC000085E003C0012B11F088E08B871E141F0410
:10BC100014F41A8604C0EF2811F081E08A87DF91BE
:10BC2000CF911F910F91FF90EF90DF90CF90BF9039
:10BC3000AF9008958F929F92AF92BF92CF92DF9272
:10BC4000EF92FF920F931F93DF93CF93CDB7DEB7A1
:10BC500028970FB6F894DEBF0FBECDBF8C01D62E4D
:10BC6000C72E7A01DC0111968C918150833028F423
:10BC7000C8010E94A25B20E0B8C0C8010A960E94D9
:10BC8000FF51F7018089A82EBB242D2D3C2DC90121
:10BC9000FC01AE014F5F5F4FB5E08B2E912C8C0EF7
:10BCA0009D1E60E070E0AFEFCA2ED12C2AC08081CB
:10BCB0001816BCF42181D80112968D919C9113978E
:10BCC000821B9109DA018D939C932281D8011496ED
:10BCD0008D919C911597821B9109D4018D939C9312
:10BCE00006C0D401CD92DC92DA01CD92DC926F5F76
:10BCF0007F4FE25BFF4F4E5F5F4F82E090E0880E28
:10BD0000991E6A157B059CF2D80111969C9111979A
:10BD100097FF0BC01A961C921A978AE01B968C9379
:10BD20001B979F5F11969C9347C094302CF0C801DD
:10BD3000B7010E94AC5C40C0F80112861386B9803E
:10BD4000AA80DD80CE804B815C81AF81B8858D2D4E
:10BD50009C2D9C01B90137FF03C0709561957F4F01
:10BD60008B2D9A2D9C0137FF03C0309521953F4FB5
:10BD7000FB01E20FF31FBD01B7FF03C07095619592
:10BD80007F4F9A0157FF03C0309521953F4F620FB7
:10BD9000731FE617F70724F0F7018089813039F423
:10BDA000C801B7014B2D5A2D2D2D3C2D03C0C801C4
:10BDB000B7019D010E944D5D89819A8105960B977F
:10BDC00010F020E007C020E08D819E8106960D973F
:10BDD00008F421E08B819C8105960B9730F48F81CC
:10BDE000988506960D9708F42260822F28960FB644
:10BDF000F894DEBF0FBECDBFCF91DF911F910F91A1
:10BE0000FF90EF90DF90CF90BF90AF909F908F907A
:10BE100008953F924F925F926F927F928F929F927E
:10BE2000AF92BF92CF92DF92EF92FF920F931F9348
:10BE3000CF93DF93582E492E7B015A0139019C0183
:10BE40006901E90100E010E073E0372E34C09C2E58
:10BE50008D2ECE01B7010E94B959F70181854C8121
:10BE60005D81480F511D57FD1BC081812A813B8197
:10BE7000280F311D37FD14C0848590E065E0880FE0
:10BE8000991F6A95E1F78417950754F0848190E033
:10BE900045E0880F991F4A95E1F7821793070CF444
:10BEA00039828981833021F0892D982D0E94855215
:10BEB0000F5F1F4F6196F501838194810817190761
:10BEC00030F28581968163E070E00E949E63892B49
:10BED000B1F010E0C0E0D0E00BC0C601B301A70193
:10BEE0000E941A5E182B219681E190E0C80ED91E9F
:10BEF000F50183819481C817D90778F310C00E9497
:10BF0000606368EE73E00E94B2638F58934034F030
:10BF1000852D942DB501A7010E94615C10E000E021
:10BF2000C12EDD241EE4B12E16EA27C0802F90E03A
:10BF300001968C219D21892BF9F00B9DE0011124A4
:10BF4000C60DD71D88811816BCF49B8191FD14C0C5
:10BF50008150888392609B831E82181644F088E18A
:10BF600060E940E00E947D3F1A83198305C087E1A4
:10BF700060E940E00E947D3F0F5FF701808908176C
:10BF8000A8F2DF91CF911F910F91FF90EF90DF907A
:10BF9000CF90BF90AF909F908F907F906F905F9069
:10BFA0004F903F900895DC0114968C9114978F5F09
:10BFB00014968C931497823098F014961C921497D0
:10BFC000AC5BBF4F8C91A454B04090E0FC01EE0FED
:10BFD000FF1FE80FF91FE050FA4F86EA8183808344
:10BFE00086EA90E05A969C938E93599758969C9324
:10BFF0008E9357979B969C938E939A9799969C9322
:10C000008E939897DC969C938E93DB97DA969C930D
:10C010008E93D9970895CF93DF93EC01DB011296AD
:10C020008C9112978C831D8211968C9111978A8323
:10C030001B821E968C911E97888317961C921797C9
:10C040008D8590E0FC01EE0FFF1FE80FF91FE05017
:10C05000FA4F8E8582831E968C91813059F0813003
:10C0600028F0823069F08330A1F40EC08C819D816C
:10C07000059603C08C819D8105979D838C8309C0A3
:10C080008A819B81039703C08A819B8103969B834E
:10C090008A83DF91CF910895AF92BF92CF92DF92C2
:10C0A000EF92FF920F931F93CF93DF93FC017B01DD
:10C0B000EA015901C480D484C801BF010E94B95962
:10C0C00030E060E070E023E04FC0FB01A4E0EE0F41
:10C0D000FF1FAA95E1F7E60FF71FEA0DFB1D81810F
:10C0E00018160CF43FC0D80114964D915C91159729
:10C0F00084819581481B590B57FF03C0509541958A
:10C100005F4F8D2D90E04817590764F5D8011296BE
:10C110004D915C91139782819381481B590B57FF76
:10C1200003C0509541955F4F8C2D90E048175907FB
:10C13000CCF48C81829FC00111248F5F81838A851A
:10C140009B8501969B878A8789858F5F89873F5F5B
:10C1500039F4B4E0CB0EE5E0DE0E60E070E002C042
:10C16000333070F46F5F7F4FD70113968D919C91A0
:10C1700014976817790708F4A8CF332309F44EC041
:10C1800086EA90E0F80193838283958384831D82FD
:10C19000D70111961C9211978985883078F08C917F
:10C1A0008C608C932FE0329F900111248A859B85AF
:10C1B000820F931F9B878A8786E12CC08330A0F073
:10C1C000F701808188608B7F8083232F30E053E0EC
:10C1D000220F331F5A95E1F78A859B85820F931FA3
:10C1E0009B878A8785E116C0823099F4D7018C91AC
:10C1F000877F84608C93232F30E0220F331F220F20
:10C20000331F8A859B85820F931F9B878A8784E1D2
:10C2100001C083E160E940E00E947D3FDF91CF9162
:10C220001F910F91FF90EF90DF90CF90BF90AF9054
:10C2300008952F923F924F925F926F927F928F92CA
:10C240009F92AF92BF92CF92DF92EF92FF920F93A5
:10C250001F93CF93DF934C012B015A013901EA015F
:10C26000CC24DD2416EA212E312C7601B4E0EE0C2C
:10C27000FF1CBA95E1F7EC0CFD1C85E190E0E80E9F
:10C28000F91EEA0CFB1CC401B201A5019301870150
:10C290000E944C608D89813059F0813028F08230C5
:10C2A00069F08330A1F40EC0898D9A8D039603C086
:10C2B000898D9A8D03979A8F898F09C08F89988D60
:10C2C000029703C08F89988D0296988F8F8B498D26
:10C2D0005A8D57FD24C06F89788D77FD20C0413D70
:10C2E0005105ECF465387105D4F46F5F7F4F4D5FF5
:10C2F0005F4FC4010E942E5A882369F06F89788DA0
:10C300006C5F7F4F498D5A8D485F5F4FC4010E941B
:10C310002E5A882321F4F5018781893020F0388E48
:10C320002F8A3A8E298EC7010E9485520894C11C1B
:10C33000D11C6196F3E0CF16D10409F096CFDF91BE
:10C34000CF911F910F91FF90EF90DF90CF90BF9012
:10C35000AF909F908F907F906F905F904F903F90A5
:10C360002F9008952F923F924F925F926F927F92FB
:10C370008F929F92AF92BF92CF92DF92EF92FF92F5
:10C380000F931F93CF93DF934C012B015A01390177
:10C39000EA01CC24DD2486EA282E312C760104E043
:10C3A000EE0CFF1C0A95E1F7EC0CFD1C85E190E01A
:10C3B000E80EF91EEA0CFB1CC401B201A5019301B1
:10C3C00087010E944C608D89813059F0813028F0BE
:10C3D000823069F08330A1F40EC0898D9A8D059664
:10C3E00003C0898D9A8D05979A8F898F09C08F898F
:10C3F000988D039703C08F89988D0396988F8F8BA4
:10C40000498D5A8D57FD20C06F89788D77FD1CC0EE
:10C41000413D5105CCF465387105B4F46F5F7F4F31
:10C420004D5F5F4FC4010E942E5A882389F06F89A7
:10C43000788D6C5F7F4F498D5A8D485F5F4FC40187
:10C440000E942E5A882321F0388E2F8A3A8E298E08
:10C45000C7010E9485520894C11CD11C619692E0CC
:10C46000C916D10409F09ACFDF91CF911F910F9196
:10C47000FF90EF90DF90CF90BF90AF909F908F9004
:10C480007F906F905F904F903F902F900895FA01AA
:10C490004481442319F0413041F404C0AF010E94AB
:10C4A000B2610895AF010E94196108950F931F931F
:10C4B000CF93DF93EC018091FA0C823040F089E158
:10C4C00060E941E00E947D3F1092FA0C03C08F5F4B
:10C4D0008093FA0C0091FA0C81E1089FC0011124AD
:10C4E00045968C0F9D1FBE010E940B6010E09801C5
:10C4F00021503040F80154E0EE0FFF1F5A95E1F74C
:10C50000E00FF11FEC0FFD1F8789908D820F931FA5
:10C51000908F878B220F331F818D928D280F391FAB
:10C52000328F218F82A190E0FC01EE0FFF1FE80FF8
:10C53000F91FE050FA4F81E48283FE01E45BFF4F74
:10C54000808181508083DF91CF911F910F91089559
:10C55000CF93DF93FC01818D928D863A910514F083
:10C5600020E006C082A593A5863A910564F121E0FA
:10C57000822F90E0EC0174E0CC0FDD1F7A95E1F79B
:10C58000C80FD91FCE0FDF1F898D9A8D863A91056E
:10C59000D1F481E1289FC001112445968E0F9F1F81
:10C5A000BF010E940B608AA190E0FC01EE0FFF1F0B
:10C5B000E80FF91FE050FA4F80E4828382E160E9DE
:10C5C00041E00E947D3FDF91CF910895DC011496F8
:10C5D0002C911497822F90E0FC01EE0FFF1FE80FC3
:10C5E000F91FEA0FFB1FE65BFF4F17969C91179709
:10C5F0008081EA54F040981788F0E75BFF4F808114
:10C60000882361F0222319F0213041F404C0CD01C8
:10C610000E94A8620895CD010E9456620895A0E08C
:10C62000B0E0E5E1F3E60C942964EC01A880B98060
:10C63000CA80DB80A114B104C104D10441F484E2B6
:10C64000A82E89EDB82E8BE5C82E87E0D82EC6011E
:10C65000B5012DE133EF41E050E00E94066427EA86
:10C6600031E440E050E00E94E7637B018C01C601A9
:10C67000B5012DE133EF41E050E00E940664CA01AC
:10C68000B9012CEE34EF4FEF5FEF0E94E7636E0DC0
:10C690007F1D801F911F97FF04C061507040804034
:10C6A0009048688379838A839B839B013F77C90184
:10C6B000CDB7DEB7EAE00C9445640E940F6308959D
:10C6C00088EA91E00E940F630895A0E0B0E08093B3
:10C6D000A8019093A901A093AA01B093AB0108957A
:10C6E0006817790768F4FB01DC01E40FF51FA40F5C
:10C6F000B51F02C002900E9241505040D8F70895E5
:10C700000C948963DC0101C06D9341505040E0F707
:10C710000895FB01DC0102C001900D924150504090
:10C72000D8F70895991B79E004C0991F961708F06F
:10C73000961B881F7A95C9F780950895AA1BBB1B85
:10C7400051E107C0AA1FBB1FA617B70710F0A61B11
:10C75000B70B881F991F5A95A9F780959095BC0132
:10C76000CD01089597FB092E07260AD077FD04D046
:10C77000E5DF06D000201AF4709561957F4F08958B
:10C78000F6F7909581959F4F0895A1E21A2EAA1B66
:10C79000BB1BFD010DC0AA1FBB1FEE1FFF1FA21771
:10C7A000B307E407F50720F0A21BB30BE40BF50B6E
:10C7B000661F771F881F991F1A9469F760957095F7
:10C7C000809590959B01AC01BD01CF010895629FBA
:10C7D000D001739FF001829FE00DF11D649FE00D79
:10C7E000F11D929FF00D839FF00D749FF00D659FDA
:10C7F000F00D9927729FB00DE11DF91F639FB00DD9
:10C80000E11DF91FBD01CF011124089597FB092EE9
:10C8100005260ED057FD04D0B8DF0AD0001C38F42E
:10C8200050954095309521953F4F4F4F5F4F08955C
:10C83000F6F790958095709561957F4F8F4F9F4F3C
:10C8400008952F923F924F925F926F927F928F92B4
:10C850009F92AF92BF92CF92DF92EF92FF920F938F
:10C860001F93CF93DF93CDB7DEB7CA1BDB0B0FB699
:10C87000F894DEBF0FBECDBF09942A883988488856
:10C880005F846E847D848C849B84AA84B984C884EC
:10C89000DF80EE80FD800C811B81AA81B981CE0FE3
:10C8A000D11D0FB6F894DEBF0FBECDBFED010895C8
:04C8B000F894FFCF2A
:10C8B4000000000000000000000000000000000074
:10C8C4000000000000000000000000000000000064
:10C8D4000000000000000000000000000000000054
:10C8E4000000000000000000000000000000000044
:10C8F4000000000000000000000000000000000034
:10C904000000000000000000000000000000000023
:10C914000000000000000000000000000000000013
:10C924000000000000000000000000000000000003
:10C9340000000000000000000000000000000000F3
:10C944004122B7252F29A72C20309A330040889103
:0CC95400D2E4ADB5B6BEBFFF010000008C
:00000001FF
